:0200000480007A
:10000000B72F0000938F0F8073900F306F00400365
:100010001300000013000000130000001300000094
:100020001300000013000000130000001300000084
:100030001300000013000000130000001300000074
:100040009702000093824211739052309300000097
:10005000130100009301000013020000930200004E
:100060001303000093030000130400009304000036
:10007000130500009305000013060000930600001E
:100080001307000093070000130800009308000006
:100090001309000093090000130A0000930A0000EE
:1000A000130B0000930B0000130C0000930C0000D6
:1000B000130D0000930D0000130E0000930E0000BE
:1000C000130F0000930F000097110200938141CF9E
:1000D0001705020013050553979503009385057DC9
:1000E00013060000EF00001A17050200130505446F
:1000F000970502009385854C13060000EF008018D9
:1001000017A503001305C57A97B503009385057AF3
:1001100037B6ABAB1306B6BAEF00C01617B1030083
:1001200013010179EF90C0009392120093D2120054
:100130009382D2FF638A02008322010013014100EF
:100140006F0000177300203083220100130141006B
:10015000730020301301C1FF23205100F32220340B
:10016000E3C402FC8322010013014100130141F8A2
:1001700023221100232421002326310023284100BB
:10018000232A5100232C6100232E71002320810299
:10019000232291022324A1022326B1022328C10293
:1001A000232AD102232CE102232EF1022320010570
:1001B0002322110523242105232631052328410567
:1001C000232A5105232C6105232E71052320810745
:1001D000232291072324A1072326B1072328C1073F
:1001E000232AD107232CE107232EF107732520347E
:1001F000F3251034130601006F000000731015344E
:1002000083204100032181008321C10003220101D9
:1002100083224101032381018323C10103240102BD
:1002200083244102032581028325C10203260103A1
:1002300083264103032781038327C1030328010485
:1002400083284104032981048329C104032A010569
:10025000832A4105032B8105832BC105032C01064D
:10026000832C4106032D8106832DC106032E010731
:10027000832E4107032F8107832FC1071301C10775
:10028000730020302320C5006376B50013054500B8
:100290006FF05FFF678000000000000000000000BA
:1002A000000000000000000000000000000000004E
:1002B000130101F8232011002322210023243100FF
:1002C0002326410023285100232A6100232C71009A
:1002D000232E8100232091022322A1022324B10294
:1002E0002326C1022328D102232AE102232CF10272
:1002F000232E010323201105232221052324310568
:100300002326410523285105232A6105232C710545
:10031000232E8105232091072322A1072324B1073F
:100320002326C1072328D107232AE107232CF1071D
:100330009702020083A2C22223A02200F3221034DB
:10034000232E5106EF00C03B17010200032141217B
:10035000032101008322C10773901234B7220000E9
:100360009382028873A00230832001000322C1001F
:100370008322010103234101832381010324C1015D
:100380008324010203254102832581020326C10241
:100390008326010303274103832781030328C10325
:1003A000832801040329410483298104032AC10409
:1003B000832A0105032B4105832B8105032CC105ED
:1003C000832C0106032D4106832D8106032EC106D1
:1003D000832E0107032F4107832F81071301010893
:1003E00073002030970202009382C22123A01200E2
:1003F00023A2220023A4320023A6420023A85200F5
:1004000023AA620023AC720023AE820023A09202D2
:1004100023A2A20223A4B20223A6C20223A8D202CC
:1004200023AAE20223ACF20223AE020323A01205A8
:1004300023A2220523A4320523A6420523A85205A0
:1004400023AA620523AC720523AE820523A092077E
:1004500023A2A20723A4B20723A6C20723A8D20778
:1004600023AAE20723ACF207EF60907317010200A2
:100470000321010F032101008322C107739012346D
:10048000B72200009382028873A00230832001000B
:100490000322C1008322010103234101832381013F
:1004A0000324C10183240102032541028325810223
:1004B0000326C10283260103032741038327810307
:1004C0000328C103832801040329410483298104EB
:1004D000032AC104832A0105032B4105832B8105CF
:1004E000032CC105832C0106032D4106832D8106B3
:1004F000032EC106832E0107032F4107832F810797
:100500001301010873002030970202009382820FCA
:1005100083A0020003A1420083A1820003A2C200C3
:1005200083A2020103A3420183A3820103A4C201A7
:1005300083A4020203A5420283A5820203A6C2028B
:1005400083A6020303A7420383A7820303A8C2036F
:1005500083A8020403A9420483A9820403AAC20453
:1005600083AA020503AB420583AB820503ACC20537
:1005700083AC020603AD420683AD820603AEC2061B
:1005800083AE020703AFC20983AF82076780000012
:1005900073700430130101F823201100232221007D
:1005A000232431002326410023285100232A6100FF
:1005B000232C7100232E8100232091022322A102EB
:1005C0002324B1022326C1022328D102232AE102D7
:1005D000232CF102232E01032320110523222105C0
:1005E000232431052326410523285105232A6105AB
:1005F000232C7105232E8105232091072322A10797
:100600002324B1072326C1072328D107232AE10782
:10061000232CF1079702020083A282F423A0220078
:10062000232E1106EF30007417010200032141F35D
:10063000032101008322C10773901234B722000006
:100640009382028873A00230832001000322C1003C
:100650008322010103234101832381010324C1017A
:100660008324010203254102832581020326C1025E
:100670008326010303274103832781030328C10342
:10068000832801040329410483298104032AC10426
:10069000832A0105032B4105832B8105032CC1050A
:1006A000832C0106032D4106832D8106032EC106EE
:1006B000832E0107032F4107832F810713010108B0
:1006C00073002030737004306F00000073104530E9
:1006D000678000007325403073F04330678000006E
:1006E00097070000938747FE232EB5FE2322C5FA05
:1006F000232635F82320F5F8130505F86780000058
:10070000130101FF23261100EF605046EF20501C1B
:10071000631805008320C1001301010167800000F8
:100720008320C100130101016F30C063930785006E
:100730001307F0FF2322F5002324E5002326F5000C
:100740002328F500232005006780000023280500EA
:10075000678000008327450023A2F50003A78700D8
:1007600023A4E50003A787002322B70023A4B70032
:1007700023A8A50083270500938717002320F500F1
:100780006780000003A605009307F0FF13078500AC
:100790006316F6006F008003138707008327470066
:1007A00083A60700E37AD6FE23A2F50023A4B700B0
:1007B00023A4E5002322B70023A8A5008327050072
:1007C000938717002320F5006780000003270501A9
:1007D000832747006FF05FFD0327450083268500D0
:1007E000832705012324D70003278500832645009E
:1007F0002322D70003A747006316A700032785001D
:1008000023A2E7002328050003A507001305F5FF31
:1008100023A0A70067800000130101FF23248100AB
:1008200023261100232291008327050413040500C9
:100830006398070283270500638C070C13050000EB
:100840008327840393871700232CF4028320C1009D
:10085000032481008324410013010101678000000B
:1008600093040600631A0604032585001386070017
:10087000EF50100C832784008326040403274400D0
:10088000B387D7002324F400E3EAE7FA83270400C0
:10089000130500002324F4008327840393871700A3
:1008A000232CF4028320C10003248100832441000F
:1008B00013010101678000000325C50013860700AE
:1008C000EF501007032704048327C4008326040085
:1008D0003307E040B387E7002326F40063F8D7002E
:1008E000832744003387E7002326E4009307200092
:1008F000E396F4F483278403E38207F483278403D5
:10090000130500009387F7FF232CF4026FF05FF3C9
:1009100003254500EF30506C232204006FF05FF296
:10092000130101FE232E1100232C8100232A9100A4
:10093000032445052326A100630E04020327840334
:100940008327C4036366F700737004306F000000F0
:1009500003278403930400006362F7028320C1012C
:100960000324810113850400832441011301010242
:1009700067800000737004306F000000138605006C
:10098000130504009305C100EFF01FE90327840459
:100990009307F0FF93040500630AF700832784049C
:1009A000938717002324F4046FF05FFB832744022E
:1009B000E38607FA13054402EF30101EE30005FA40
:1009C000930410006FF09FF9032605049387050038
:1009D000630406028325C50003274500B385C500CF
:1009E0002326B50063E6E500832505002326B50030
:1009F000138507006F50C07367800000130101FD6D
:100A000023248102232611021304050023229102CC
:100A100023202103232E3101232C4101232A5101BC
:100A2000EF30906883278404635CF004130A440267
:100A30009309F0FF1309100083244405638E04001A
:100A400003A7840383A7C403232681006368F70AEE
:100A5000737004306F000000832744026382070232
:100A600013050A00EF3050136314050C8327840428
:100A70009387F7FF2324F40483278404E34EF0FADA
:100A80009307F0FF2324F404EF305065EF30D0617A
:100A900083274404635CF002832704016388070210
:100AA0009304040113850400EF30100F631605084A
:100AB000832744049387F7FF2322F4048327440405
:100AC0006356F00083270401E39E07FC9307F0FFC1
:100AD0002322F404EF3090608320C10203248102BA
:100AE00083244102032901028329C101032A8101D0
:100AF000832A4101130101036780000003A78403D7
:100B0000E376F7F6130600009305C1001385040091
:100B1000EFF09FD083A78404930A05006382370314
:100B200083A784049387170023A4F404E3902AF591
:100B3000EF30D0336FF09FF3EF3050336FF05FF74B
:100B400083A74402E38407FE13854402EF30D004F8
:100B5000E30E05FC6FF0DFFD630A0508130101FEDB
:100B6000232C810013040500232E1100232A910059
:100B7000232821012326310113890500EF30D052AB
:100B8000832404048325C4038329040013850400FB
:100B9000EF8040341307F0FF232C0402B307954085
:100BA000B387F9003385A9002322E4042322A4009B
:100BB000232434012326F4002324E404631C0902C3
:100BC0008327040163920704EF3050518320C10151
:100BD0000324810183244101032901018329C100E8
:100BE00013051000130101026780000073700430C8
:100BF0006F00000013050401EFF05FB3130544021A
:100C0000EFF0DFB26FF05FFC13050401EF30C07846
:100C100093071000E31AF5FAEFF09F976FF0DFFAF1
:100C200063160500737004306F000000130101FEAD
:100C3000232A91002328210123263101232E11008C
:100C4000232C8100930405001389050093090600F5
:100C50006382050AEF80002813059505EF50C02C2C
:100C6000130405006300050A930785052320F5009A
:100C7000232E940223202405EF3010438324040400
:100C80008325C4030329040013850400EF80802416
:100C90009306F0FF232C0402B30795403307A90005
:100CA000B307F9002322D4042322E4002326F4000E
:100CB0002324D4041305040123242401EFF01FA7E7
:100CC00013054402EFF09FA6EF305041230834058E
:100CD000232A0404130504008320C1010324810195
:100CE00083244101032901018329C1001301010269
:100CF0006780000013058005EF50002313040500F2
:100D000063160500737004306F0000002320840018
:100D10006FF01FF6130101FD2322910293040500D9
:100D20001305800523248102232611022320210399
:100D3000232E3101232C4101EF50001F1304050025
:100D400063080506232C05029307F0FF2322F50410
:100D500013071000130A05012324F40413050A00E5
:100D6000232EE40223220400232004002324040071
:100D7000232604002320040423089404232A0404C3
:100D8000EFF0DF9A1309440213050900EFF01F9AF0
:100D90008327040423220100638E0702737004304A
:100DA0006F00000013050400EFF05FC5EF20C0578F
:100DB000130504008320C10203248102832441021D
:100DC000032901028329C101032A810113010103BF
:100DD00067800000EF30900D631605008327410007
:100DE00063980710EF30502C032784038327C40334
:100DF000930400009309F0FF6362F7088327410022
:100E0000638E070A6396040013058100EF30807338
:100E1000EF30D02CEF20C01DEF3010298327440481
:100E200063943701232204048327840463943701E5
:100E300023240404EF30902A930541001305810018
:100E4000EF304073E31005F6EF30102603278403DC
:100E50008327C4036308F706EF3050281305040006
:100E6000EFF0DFB9EF20404C93041000EF30D023B7
:100E7000032784038327C403E372F7F803260404DB
:100E8000631C060683270400638A070A1305000013
:100E9000832784030327440593871700232CF40238
:100EA000630607089305000013050400EFF05FA731
:100EB000930710006314F500EFF08FEDEF30102270
:100EC0006FF01FEFEF3090218325410013050A00DA
:100ED000EF30801F13050400EFF05FB2EF20C04435
:100EE000E31405F8EFF0CFEA930410006FF01FF859
:100EF000737004306F000000032584009305000028
:100F0000EF50002383278400832604040327440032
:100F1000B387D7002324F400E3EAE7F6832704002D
:100F2000130500002324F4006FF09FF6832744028A
:100F3000639E0700E30405F86FF01FF803254400E3
:100F4000EF309009232204006FF09FF4130509008D
:100F5000EF30804493071000E312F5F66FF0DFF5F1
:100F600063160500737004306F0000006376B500EF
:100F7000737004306F000000130101FF232481000F
:100F8000130620001384050093050000232611009A
:100F9000EFF01FC9630C0500232C85028320C100DC
:100FA0000324810013010101678000007370043085
:100FB0006F000000130101FC232E1102232C81027B
:100FC000232A9102232821032326310323244103CA
:100FD00023225103232061032326C1006304051645
:100FE000638A051493072000639CF6000327C5035A
:100FF000930710006306F700737004306F00000061
:10100000938406001389050013040500EF30006A7D
:10101000631A05008327C1006386070073700430DC
:101020006F000000EF305008032784038327C403B8
:1010300093090000130B2000130AF0FF930A040128
:101040006364F708638464118327C100638C071C01
:101050006396090013058101EF30C04EEF30100890
:10106000EF101079EF305004832744046394470154
:101070002322040483278404639447012324040463
:10108000EF30D0059305C10013058101EF30804E8C
:1010900063100518EF305001032784038327C4032E
:1010A0006304F706EF30900313050400EFF01F957B
:1010B000EF20802793091000EF30007F032784037F
:1010C0008327C403E370F7F80326040463040608C7
:1010D000639004160325840093050900EF50400532
:1010E000832784008326040403274400B387D700A2
:1010F0002324F40063E4E7068327040013050000BB
:101100002324F4006F00C005EF30407D8325C1002B
:1011100013850A00EF20507B13050400EFF01F8EAB
:10112000EF208020E31805F8EFF08FC69309100038
:101130006FF09FF883270504E38607EA7370043095
:101140006F000000737004306F0000000326040479
:101150006314060683270400638C07101305000040
:10116000832784030327440593871700232CF40265
:101170006306070E9385040013050400EFF04FFA91
:10118000930710006302F50EEF3040751305100051
:101190008320C10303248103832441030329010322
:1011A0008329C102032A8102832A4102032B0102FF
:1011B00013010104678000000325C40093050900A2
:1011C000EF401077832704040327C400832604001C
:1011D000B307F0403307F7002326E400637CD70011
:1011E00003274400B307F7002326F40093072000E9
:1011F000E396F4F683278403E38207F683278403C8
:10120000130500009387F7FF232CF4026FF05FF5BE
:1012100013050400EFF08FFEEF200011130500000E
:101220006FF01FF7EF30806B130500006FF05FF673
:101230000325C40093050900EF40906F8327040441
:101240000327C40083260400B307F0403307F700E8
:101250002326E400E37CD7F86FF09FF8832744024D
:1012600063900702E30205F2EFF08FB26FF0DFF157
:1012700003254400EF304056232204006FF05FEE58
:1012800013054402EF30401193071000E31EF5EE02
:101290006FF09FFD63040504130101FF2324810007
:1012A0002322910023261100232021010329450038
:1012B00013040500EF30803E930400006304A9028C
:1012C0008320C10003248100138504000329010049
:1012D0008324410013010101678000007370043012
:1012E0006F0000008327C400930410009387F7FF6A
:1012F0002326F400E39607FC930600001306000083
:101300009305000013050400EFF0DFCA6FF05FFBE8
:101310006302050A63880508130101FE232C81007E
:10132000232A91002328210123244101232E110087
:101330002326310193072000938406001309060039
:10134000138A050013040500639CF6000327C503F8
:10135000930710006302F70A737004306F000000F7
:10136000EFF04FB7032784038327C40393090500D5
:101370006366F7049304000013850900EFF00FB5CE
:101380008320C10103248101138504000329010185
:10139000832441018329C100032A81001301010232
:1013A0006780000083270504E38807F67370043024
:1013B0006F000000737004306F0000000326040407
:1013C000631E060C832704006388071283278403A7
:1013D0001307F0FF93871700232CF402832784045C
:1013E0006388E70E83278404930410009387170013
:1013F0002324F4046FF05FF8EFF0CFAD03278403EC
:101400008327C403930905006360F70603260404D9
:10141000E30A06FA0325C40093050A00EF40505181
:10142000832704040327C40083260400B307F04085
:101430003307F7002326E4006378D700032744002E
:10144000B307F7002326F40093072000E390F4F895
:1014500083278403E38C07F6832784039387F7FFAE
:10146000232CF4026FF09FF603260404E30C06F429
:101470000325C40093050A00EF40904B8327040422
:101480000327C40083260400B307F0403307F700A6
:101490002326E400E364D7FA6FF09FFBE39C04F695
:1014A0000325840093050A00EF40904883278400B9
:1014B0008326040403274400B387D7002324F400C1
:1014C000E3E6E7F0832704002324F4006FF01FF025
:1014D00083274405638A07029385040013050400EB
:1014E000EFF00FC493041000E31895E8E30609E851
:1014F000232099006FF05FE803254400EF30C02DF2
:10150000232204006FF09FEC832744029304100011
:10151000E38407E613054402EF201068E31805FC96
:101520006FF09FE56302050A8327050463860700C1
:10153000737004306F00000083270500638A07087A
:10154000130101FE232C8100232A910013040500BE
:101550002328210123263101232E110013890500A0
:10156000EFF04F97032784038327C40393090500F3
:10157000930400006376F702832784031307F0FFC8
:1015800093871700232CF40283278404638AE704DB
:101590008327840493041000938717002324F40402
:1015A00013850900EFF08F928320C101032481018C
:1015B0001385040003290101832441018329C1000B
:1015C0001301010267800000737004306F00000097
:1015D00083274500E38607F6737004306F00000030
:1015E0008327440563800702930500001305040068
:1015F000EFF00FB3930710006300F502930410009F
:101600006FF01FFA83274402E38A07FE13054402A2
:10161000EF209058E30405FEE30209FE9307100053
:101620002320F9006FF09FFD130101FC232E11020E
:10163000232C8102232A910223282103232631030C
:10164000232441032326C100630005166386051485
:10165000938906001389050013040500EF30000587
:10166000631A05008327C100638607007370043086
:101670006F000000EF30402383278403639E070A36
:101680008327C1006388071813058101EF20906B41
:101690009304F0FF130A44026F008002EF3000242D
:1016A00013050400EFF08FB5EF101048EF30C01FA6
:1016B00083278403639207088327C100638C071480
:1016C000EF30C021EF10D012EF30001E832744040A
:1016D000639497002322040483278404639497006F
:1016E00023240404EF30801F9305C10013058101FA
:1016F000EF20506863160510EF30001B832784032A
:10170000E39E07F8EF30801D832704006386070AF5
:101710008325C10013050A00EF20101B13050400E8
:10172000EFF0CFADEF10504063040508EF30C01765
:1017300083278403E38207F8930509001305040057
:101740008324C400EFF04FA8639209088327840321
:10175000032704009387F7FF232CF4026316070086
:10176000EF30001F2322A4008327040163900708A1
:10177000EF30C016130510008320C103032481033A
:1017800083244103032901038329C102032A81021F
:10179000130101046780000083270504E38A07EA38
:1017A000737004306F000000737004306F0000002D
:1017B000EFE01FDE6FF09FF7EF30000F03254400CE
:1017C000EF209071EF3080116FF09FF48327440277
:1017D00023269400E38E07F813054402EF20D03B44
:1017E000E30805F8EFE0DFDA6FF09FF81305040176
:1017F000EF20903A93071000E31CF5F66FF09FFE80
:1018000013050400EFF08F9FEF1010321305000056
:101810006FF09FF6EF30800C130500006FF0DFF5DE
:1018200063000506130101FF232481002320210109
:1018300023261100232291008324450013890500EB
:1018400013040500EF2090656380A4049306000054
:10185000130609009305000013050400EFF0DFDC18
:1018600093071000630CF5028320C100032481005C
:101870008324410003290100130101016780000056
:10188000737004306F0000008327C400130510003C
:10189000938717002326F4006FF01FFD8327C400F1
:1018A000938717002326F4006FF01FFC63080506DA
:1018B0006386050C130101FE232C8100232A91006D
:1018C000232821012326310123244101130405008B
:1018D000232E11001309060093890500EFE09FDF16
:1018E00083278403130A050093040000639C070206
:1018F00013050A00EFE09FDD8320C101032481016D
:101900001385040003290101832441018329C100B7
:10191000032A810013010102678000007370043004
:101920006F00000003260404630406028325C4003C
:1019300083274400B385C5002326B40063E6F50081
:10194000832504002326B40013850900EF40407E60
:10195000832784031307F0FF9387F7FF232CF402F8
:10196000832744046384E70283274404930410001C
:10197000938717002322F4046FF09FF78327050451
:10198000E38A07F2737004306F00000083270401BC
:1019900063960700930410006FF09FF51305040190
:1019A000EF20901FE30805FEE30609FE93071000F1
:1019B0002320F9006FF01FFE630605088327050446
:1019C000638A050863840708130101FE232C810044
:1019D000232A910023282101232441011304050017
:1019E000232E110023263101138A0500EFE09FCE3C
:1019F000832784031309050093040000638E070006
:101A00008329C40093050A0013050400EFE0DFFBFF
:101A1000930410002326340113050900EFE01FCBC7
:101A20008320C101032481011385040003290101DE
:101A3000832441018329C100032A8100130101028B
:101A400067800000737004306F0000007370043012
:101A50006F000000E38C07FE737004306F0000001D
:101A600063160500737004306F000000130101FF5E
:101A7000232481001304050023261100EF20D062E7
:101A800003248403EF2090658320C1001305040024
:101A90000324810013010101678000006316050023
:101AA000737004306F000000130101FF2326110042
:101AB0002324810013040500EF20105F8327840393
:101AC0000324C4033304F440EF20506113050400E1
:101AD0008320C100032481001301010167800000FD
:101AE00063060500032585036780000073700430DA
:101AF0006F00000063080504978703009387C7D62B
:101B000003A747006304E50403A7C7006302E508D1
:101B100003A74701630AE50603A7C7016302E506B9
:101B200003A74702630AE50403A7C7026302E504AB
:101B300003A74703630AE50203A7C7036302E5029D
:101B40006F408056737004306F0000001307000070
:101B500013173700B387E70023A007006F40C05476
:101B6000130770006FF0DFFE130760006FF05FFE79
:101B7000130750006FF0DFFD130740006FF05FFDAB
:101B8000130730006FF0DFFC130720006FF05FFCDD
:101B9000130710006FF0DFFB0325C504678000000A
:101BA0002326B50467800000034505056780000013
:101BB00063080500032585031335150067800000C1
:101BC000737004306F000000630C050083278503E9
:101BD0000325C5033305F540133515006780000064
:101BE000737004306F000000978703009387C7C7A6
:101BF00003A707006300070403A78700630807041F
:101C000003A707016308070403A787016308070404
:101C100003A707026308070403A7870263080704F2
:101C200003A70703630C070403A7870363040704E0
:101C3000678000001307000013173700B387E70021
:101C400023A0B70023A2A70067800000130710009D
:101C50006FF09FFE130720006FF01FFE1307300088
:101C60006FF09FFD130740006FF01FFD130750003A
:101C70006FF09FFC130770006FF01FFC13076000EC
:101C80006FF09FFB97870300938707BE03A747006A
:101C90006300E50403A7C7006306E50403A7470143
:101CA0006306E50403A7C7016306E50403A747022B
:101CB0006306E50403A7C7026306E50403A7470319
:101CC000630AE50403A7C7036302A7046780000053
:101CD0001307000013173700B387E70023A007009E
:101CE00067800000130710006FF0DFFE130720006D
:101CF0006FF05FFE130730006FF0DFFD1307400049
:101D00006FF05FFD130750006FF0DFFC13077000EA
:101D10006FF05FFC130760006FF0DFFB130101FD44
:101D2000232481022322910223202103130405008E
:101D300023261102232E3101232C4101232A510194
:101D40009384050013090600EF201036032744048E
:101D50009307F0FF6314F70023220404032784048D
:101D60009307F0FF6314F70023240404EF201037D7
:101D700083278403639A07001306090093850400F0
:101D800013054402EF208050EF2010328327840493
:101D9000635CF004130A44029309F0FF1309100076
:101DA00083244405638E040003A7840383A7C4032C
:101DB000232681006368F70A737004306F00000007
:101DC000832744026382070213050A00EF20C05CE8
:101DD0006314050C832784049387F7FF2324F404FA
:101DE00083278404E34EF0FA9307F0FF2324F404DE
:101DF000EF20D02EEF20502B83274404635CF002A9
:101E000083270401638807029304040113850400F7
:101E1000EF20805863160508832744049387F7FF53
:101E20002322F404832744046356F000832704012B
:101E3000E39E07FC9307F0FF2322F404EF20102A0F
:101E40008320C10203248102832441020329010269
:101E50008329C101032A8101832A4101130101035E
:101E60006780000003A78403E376F7F613060000FB
:101E70009305C10013850400EFE01F9A83A7840433
:101E8000930A05006382370383A7840493871700AE
:101E900023A4F404E3902AF5EF20407D6FF09FF334
:101EA000EF20C07C6FF05FF783A74402E38407FE56
:101EB00013854402EF20404EE30E05FC6FF0DFFD7A
:101EC00063160500737004306F000000130101FFFA
:101ED0002322910093040500131525001305950591
:101EE000232481002326110023202101EF40C00379
:101EF0001304050063080508930785052320F500F2
:101F0000930740002320F504232E9502EF20D019DB
:101F1000832404048325C4030329040013850400D7
:101F2000EF60507B9306F0FF232C0402B30795402B
:101F30003307A900B307F9002322D4042322E400C5
:101F40002326F4002324D4041305040123242401AC
:101F5000EFE0CFFD13054402EFE04FFDEF20101836
:101F600023080404232A0404130504008320C10069
:101F7000032481008324410003290100130101018E
:101F800067800000737004306F000000130101FFD0
:101F90002324810023229100232021011304050022
:101FA0002326110013890500EF2010108327440514
:101FB0009304000063820702EF2050128320C100C7
:101FC00003248100138504000329010083244100B8
:101FD000130101016780000083278403930400003C
:101FE000E39C07FC232A2405930410006FF0DFFC18
:101FF000832745056388B700930700001385070012
:10200000678000000327850393070000E31807FE9D
:10201000130101FF2324810013040500232611006E
:10202000EF209008232A0404EF20500B8320C100E6
:102030000324810093071000138507001301010199
:1020400067800000130101FE13860500930600005F
:102050009305C100232E110023260100EFF0CFDCF1
:102060008320C1010325C100130101026780000024
:10207000130101FE232E1100232C8100232A91003D
:1020800023260100630C050213040500EFE08FE432
:1020900083278403930405006396070213850400D5
:1020A000EFE0CFE28320C101032481010325C100B9
:1020B0008324410113010102678000007370043022
:1020C0006F00000003260404630406028325C40095
:1020D00083274400B385C5002326B40063E6F500DA
:1020E000832504002326B4001305C100EF404004FB
:1020F000832784031307F0FF9387F7FF232CF40251
:1021000083274404638AE7008327440493871700E6
:102110002322F4046FF09FF883270401E38007F87B
:1021200013050401EF2040276FF05FF763020504F9
:10213000130101FD232E3101232C4101232611021D
:10214000138A0700232481022322910223202103E2
:10215000232A51012328610123267101930790004E
:102160009309070063FAE700737004306F00000002
:10217000737004306F000000130B0500938405009A
:1021800013090600938B0600930A08006302082CCB
:1021900013050006EF305059130405006302052AA9
:1021A0001319290023285503130609009305500A23
:1021B00013850A00EF40C00903C704008327040306
:1021C0001309C9FF230AE40203C704003389270166
:1021D0001379C9FF6306070E83C71400A30AF4022C
:1021E00083C71400638E070C83C72400230BF402FB
:1021F00083C724006386070C83C73400A30BF40253
:1022000083C73400638E070A83C74400230CF4029B
:1022100083C744006386070A83C75400A30CF402F3
:1022200083C75400638E070883C76400230DF4023C
:1022300083C764006386070883C77400A30DF40294
:1022400083C77400638E070683C78400230EF402DD
:1022500083C784006386070683C79400A30EF40235
:1022600083C79400638E070483C7A400230FF4027E
:1022700083C7A4006386070483C7B400A30FF402D6
:1022800083C7B400638E070283C7C4002300F4042D
:1022900083C7C4006386070283C7D400A300F40485
:1022A00083C7D400638E070083C7E4002301F404CE
:1022B00083C7E4006386070083C7F400A301F40426
:1022C000930A440013850A00A3010404232634035F
:1022D00023283405232A0404EFE04FC713058401A3
:1022E000EFE0CFC69307A000B3873741232C040447
:1022F00023288400232CF4002322840223220404B4
:10230000232E040413860B0093050B00130509000C
:10231000EFE00FBD2320A40063040A0023208A00FD
:102320007370043017E901001309C92183270900DC
:1023300097E401009384C422638C070003A7040080
:1023400083A7040083274704938717002322F704F9
:1023500017E701001307C71F83270700938717009C
:1023600097E6010023A6F61E83A70400638E070EDE
:102370008327090017EB0100130B8B30639C0700C8
:1023800083A7040083A7C70263E6F90097E701006B
:1023900023A8871C97E701009387C71983A7070025
:1023A00017E701001307471A0325C4020327070094
:1023B0009387170097E6010023AEF6162324F40452
:1023C0006376A70097E7010023A0A71893054001B3
:1023D000EF60503093850A003305AB00EFE08FB714
:1023E000832709006388070083A7040083A74704A5
:1023F000639C07088327090013041000638A070001
:1024000083A7040083A7C70263F43701EFE04F9866
:10241000130504008320C1020324810283244102A6
:10242000032901028329C101032A8101832A410171
:10243000032B0101832BC1001301010367800000FE
:1024400013850A00EF3050461304F0FF6FF05FFC75
:1024500013152600EF30502D930A0500E31A05D21C
:102460001304F0FF6FF0DFFA97E7010023AA870E4D
:102470000327070093071000630AF70217EB010018
:10248000130B0B206FF01FF103A7040083A60400B9
:10249000832747049387F7FF2322F70483A7460483
:1024A000E39A07F4736004306FF0DFF4130A00005E
:1024B00017EB0100130BCB1C930BA00013050A00B4
:1024C00093054001EF601021130A1A003305AB0099
:1024D000EFE0CFA5E3147AFF97EB0100938BCB26B7
:1024E00013850B00EFE08FA417EA0100130A0A27F7
:1024F00013050A00EFE08FA317E501001305452738
:10250000EFE0CFA217E501001305C527EFE00FA20A
:1025100017E5010013054528EFE04FA197E70100FB
:1025200023AE770397E7010023A847036FF09FE6E8
:10253000130101FF2324810023261100232291008F
:1025400023202101130405007370043097E4010077
:10255000938444FF83A70400639E0710631804005C
:1025600097E701009387C7FF03A4070013094400FE
:1025700013050900EFE04FA6832784026386070056
:1025800013058401EFE04FA59305090017E501004D
:102590001305451FEFE00F9C97E70100938787FB2A
:1025A00003A7070097E701009387C7F883A70700F1
:1025B0001307170097E6010023AEE6F803A704000F
:1025C0009387170097E6010023A6F6F6630C070031
:1025D00097E701009387C7F803A70700032747047D
:1025E000631C070E83A70400638A070697E70100B0
:1025F000938707F703A707006302871073700430FF
:1026000003A704006318070817E70100130707F57D
:102610008326070083A606006392060A1307F0FFCD
:1026200097E6010023A6E6F003A70400630807026B
:1026300003A70700032747046302070203A7070055
:1026400083A60700832747049387F7FF2322F70415
:1026500083A7460463940700736004308320C1009D
:102660000324810083244100032901001301010197
:102670006780000097E70100938787EE03A70700B4
:1026800083A7070083274704938717002322F704B3
:102690006FF0DFEC83A6070003A7070003A746043B
:1026A0001307170023A2E60417E70100130707EB3F
:1026B0008326070083A60600E38206F603270700A9
:1026C0000327C7000327C7000327470097E6010039
:1026D00023A0E6E66FF05FF503A7070083A60700D7
:1026E000832747049387F7FF2322F70483A7460431
:1026F000E39A07EE736004306FF0DFEE97E70100B6
:102700009387C7E283A707006386070073700430CE
:102710006F000000032481008320C1008324410056
:1027200003290100130101016FD09FE66304050C2A
:1027300017E701001307C7E283260700930700008D
:102740006386A60A130101FF2326110023248100BA
:10275000232291007370043097E60100938686DE91
:1027600083A70600638C0700032607008327070062
:1027700083274604938717002322F60483A70600C5
:10278000930405000324450163880700832707009D
:1027900083A747046394070697E70100938707DC44
:1027A00083A70700638C870697E701009387C7DA42
:1027B00083A707006384870697E701009387C7FD17
:1027C0006306F40497E701009387C7FB630CF402E8
:1027D000930710008320C10003248100832441005B
:1027E00013850700130101016780000013850700AE
:1027F00067800000737004306F000000EF6090038A
:102800006FF09FF9930740006FF0DFFC83A784020D
:1028100093B71700938727006FF0DFFB9307200023
:102820006FF05FFB7370043097E70100938787D1E7
:1028300003A70700631607026304050483A70700C4
:102840000325C502638C070097E70100938747D1F2
:1028500003A7070003274704631C070267800000E3
:1028600017E701001307C7CF8326070003270700D8
:1028700003A746041307170023A2E604E31005FC90
:1028800017E701001307C7CD032507006FF01FFBF3
:1028900003A7070083A60700832747049387F7FF52
:1028A0002322F70483A74604E39A07FA73600430EF
:1028B00067800000130101FF232481001304050039
:1028C00023261100EFD01FE16318040097E70100F1
:1028D000938707C903A407000324C402EFD01FDFB6
:1028E0008320C100130504000324810013010101AA
:1028F000678000009307900063F6B70073700430A0
:102900006F000000130101FE232C8100232E110013
:10291000232A910023282101232631012324410168
:10292000130405007370043017E90100130989C10D
:1029300083270900639207106300041283270405AC
:10294000638EF50A17E70100130787C163F0B7022A
:1029500083260700638E8612032707008324C7029D
:10296000B3B4950093C414006F00000183240700E2
:10297000B384844093B414000327C4026386E70E33
:10298000832784012328B40463C807009307A000A9
:10299000B385B740232CB40093172700B387E70013
:1029A0000327440197E90100938989CD9397270074
:1029B000B387F9006310F704130A440013050A00F3
:1029C000EFD09FE197E70100938707B80325C40282
:1029D00083A7070063F6A70097E7010023A6A7B621
:1029E00093054001EF60004F93050A003385A9006D
:1029F000EFD05FD663840400EFD09FB9832709002E
:102A0000638C070097E70100938787B583A70700CA
:102A100083A74704639E07048320C1010324810127
:102A200083244101032901018329C100032A810074
:102A3000130101026780000097E70100938747B206
:102A400003A7070083A7070083274704938717007E
:102A50002322F704E31404EE97E70100938747B0BD
:102A600003A407006FF09FED2326B4026FF05FF11F
:102A7000032481018320C101832441010329010131
:102A80008329C100032A8100130101026F60805A6B
:102A9000930400006FF05FEE630A0508130101FE66
:102AA000232A910097E40100938484AB83A7040058
:102AB000232E1100232C81002328210123263101FC
:102AC0006388A7047370043017E90100130989A70C
:102AD00083270900638C070003A7040083A7040071
:102AE00083274704938717002322F7040327450110
:102AF00097E70100938747CA630EF702832709000F
:102B00006388070083A7040083A74704639E070820
:102B10008320C10103248101832441010329010190
:102B20008329C10013010102678000007370043023
:102B30006F0000008327850217E70100130747C3D2
:102B4000E38EE7FAE39C07FA9309450013040500B6
:102B500013850900EFD05FC897E701009387C79EF0
:102B60000325C40283A7070063F6A70097E70100C7
:102B700023ACA79C93054001EF60C03597E70100A7
:102B8000938707B03385A70093850900EFD09FBCDA
:102B900083A704000327C40283A7C702E360F7F6F4
:102BA000EFD01F9F6FF09FF5032481018320C101A7
:102BB00083244101032901018329C100130101027A
:102BC0006F60404763020506130101FE232C81005C
:102BD000232A91002326310113040500232E11001E
:102BE00023282101EFD01FAF0327440197E70100FD
:102BF000938787BA9309050093040000630AF702DC
:102C000013850900EFD09FAC8320C101032481010B
:102C10001385040003290101832441018329C10094
:102C20001301010267800000737004306F00000020
:102C30008327840217E50100130585B3E382A7FC0F
:102C4000E39007FC97E701009387478E83A707006F
:102C50006394070697E701009387879083A707008F
:102C60008324C4021309440083A7C7021305090083
:102C7000B3B4F400EFD05FB697E701009387C78C39
:102C80000325C40283A7070093C4140063F6A700BA
:102C900097E7010023AAA78A93054001EF608023EC
:102CA00097E701009387C79D930509003385A70027
:102CB000EFD05FAA6FF0DFF493058401EFD09FA9F6
:102CC0006FF01FF4130101FE37150000232E1100D1
:102CD000232C8100232A910023282101232631015E
:102CE000232441012322510123206101EF30C0231D
:102CF000630805229304050013050006EF30C02287
:102D00001304050063040526371600009305500AD6
:102D10002328950213850400EF3080538324040395
:102D2000B71700009387C7FFB384F400B7474C453B
:102D300093879744130A4400232AF40213050A00D8
:102D4000230C0402A3010404232604022328040400
:102D5000232A0404EFD09F9F13058401EFD01F9F07
:102D60009307A000232C040493F4C4FF23288400B9
:102D7000232CF4002322840223220404232E04049F
:102D800013060000971500009385C5EA138504001B
:102D9000EFD01F952320A4007370043017D90100D1
:102DA0001309497A8327090097D401009384447B4F
:102DB000638C070003A7040083A70400832747044C
:102DC000938717002322F70417D7010013074778CA
:102DD000832707009387170097D6010023AAF6766A
:102DE00083A704006388070A8327090097E9010085
:102DF00093890989639C070083A7040083A7C702FE
:102E00006396070097D7010023AC877497D701001A
:102E10009387477203A7070097D601009386C6726F
:102E20008327C40283A606001307170017D60100E4
:102E30002322E6702324E40463F6F60017D701008A
:102E40002324F770139527003305F500131525008B
:102E500093050A003385A900EFD0DF8F832709008F
:102E60006388070083A7040083A74704639E070CB9
:102E7000832709006384070083A70400EF2050071D
:102E800093071000630AF510631C05087370043083
:102E90006F00000097D7010023A4876C0327070069
:102EA0009307100097D901009389897DE310F7F605
:102EB000938A090017EB0100130B0B8913850A0095
:102EC000938A4A01EFD09F86E31A5BFF17E5010062
:102ED00013058587EFD09F8597EA0100938A0A88BA
:102EE00013850A00EFD09F8417E50100130545887C
:102EF000EFD0DF8317E501001305C588EFD01F83EE
:102F000017E5010013054589EFD05F8297D70100CF
:102F100023A6676597D7010023A057656FF01FEFC1
:102F20008320C1010324810183244101032901017C
:102F30008329C100032A8100832A4100032B010059
:102F4000130101026780000003A7040083A60400A8
:102F5000832747049387F7FF2322F70483A74604B8
:102F6000E39807F0736004306FF09FF00324810151
:102F70008320C101032901018329C100032A8100A3
:102F8000832A4100032B010013850400832441019F
:102F9000130101026F304011737004309307F0FF8A
:102FA00017D701002326F7580324810197D7010082
:102FB00023AAA7588320C1018324410103290101C9
:102FC0008329C100032A8100832A4100032B0100C9
:102FD00097D7010023AC0756130101026FD08FC0B1
:102FE0007370043097D7010023AE07546FD0CFD150
:102FF00017D701001307875383270700938717000C
:103000002320F700678000007370043097D7010019
:103010009387475303A707006318070217D70100D8
:103020001307C7520325070083A70700638C070017
:1030300097D701009387C75203A7070003274704C8
:10304000631407026780000017D701001307475178
:10305000832607000327070003A74604130717006A
:1030600023A2E6046FF09FFB03A7070083A60700D7
:10307000832747049387F7FF2322F70483A7460497
:10308000E39207FC7360043067800000130101FFC6
:103090002326110023248100EFD0CFE397D701002E
:1030A0009387C74A03A40700EFD04FE28320C100F3
:1030B000130504000324810013010101678000004F
:1030C00097D701009387C74803A5070067800000D2
:1030D000130101FD232611022324810223229102E0
:1030E00023202103232E3101232C4101232A5101C6
:1030F000232861012326710197D701009387074395
:1031000083A70700639A070617D701001307074430
:10311000832707009387170097D6010023A8F6425C
:10312000832A0700638A0A0A97D7010093874740DA
:1031300083A707009304000063FEFA0A97D90100F1
:103140009389095417DA0100130A8A4183270A0078
:103150009306100003A7C70293172700B387E70061
:1031600093972700B389F90083A7090063F4F60257
:10317000930410006F00000297D701009387473C2B
:1031800083A70700930400009387170017D7010057
:103190002328F73A97D701009387473A83A7070078
:1031A00063840700930410008320C102032481027A
:1031B0001385040003290102832441028329C101EC
:1031C000032A8101832A4101032B0101832BC100C2
:1031D000130101036780000017D4010013040438B1
:1031E0008327040083A707006388070C73700430EB
:1031F0006F00000017D401001304443697D9010072
:103200009389094817DA0100130A8A3517DB010090
:10321000130B8B338327040083A707006380070801
:103220008327040083A7C70003A9C7008327490099
:10323000930B490013850B0063EAFA06EFD0CFD950
:10324000832789021305890163840700EFD0CFD853
:103250008327C90203270B0093850B0013952700D2
:103260003305F500131525003385A9006376F700B3
:1032700017D70100232AF72CEFD0CFCD83270A00E0
:103280000327C90283A7C702E366F7F88327040070
:103290009304100083A70700E39407F89307F0FF57
:1032A00017D701002326F7286FF05FEA17D7010030
:1032B0002320F7286FF09FE917D701001307C729CC
:1032C000832704000327070097D6010023A8E628D8
:1032D00017D701002322F72897D701009387C72526
:1032E00083A707009387170017D701002326F72429
:1032F0008327040083A70700639A07009307F0FF62
:1033000017D701002326F7226FF01FE2832704005E
:1033100083A7C70083A7C70083A7470017D701006B
:103320002328F7206FF05FE097D7010093870720ED
:1033300003A7070063160700737004306F000000D6
:10334000130101FE232E1100232C8100232A91005A
:103350002328210123263101232441012322510165
:10336000232061017370043097D401009384841D7D
:1033700003A704006310071203A707001307F7FF52
:1033800097D6010023A4E61A83A70700639E070AC5
:1033900097D701009387C71B83A707006386070A97
:1033A00097DA0100938ACA2D17DA0100130ACA19A5
:1033B00017D901001309C91A930910006F00C00141
:1033C0003385EA00EFD00FB9832709000327C40231
:1033D00083A7C7026374F70683A70A0F6380070EEB
:1033E00083A7CA0F03A4C70013058401EFD0CFBE83
:1033F000130B440013050B00EFD00FBE8327C4024C
:1034000083260A0093050B00139527003305F5006A
:1034100013152500130705003385AA00E3F2F6FA19
:1034200017D701002322F712EFD0CFB2832709006C
:103430000327C40283A7C702E360F7FA97D7010006
:1034400023AE370F6FF05FF91304000083A7040069
:10345000638C070097D701009387871083A7070025
:1034600083A7470463980704130504008320C10160
:103470000324810183244101032901018329C1001F
:10348000032A8100832A4100032B0100130101025A
:103490006780000017D701001307870C83260700F9
:1034A0000327070003A746041307170023A2E60417
:1034B0006FF09FECEF5010386FF01FFB17D4010036
:1034C0001304040883270400638C07028327040085
:1034D0001309100063860702EFF09FBF6306050023
:1034E00097D7010023AC2705832704009387F7FFB4
:1034F00017D701002326F70483270400E39E07FC67
:1035000097D701009387870303A70700930710004D
:10351000E31CF7F2EFD0CF87130410006FF01FF316
:103520006304050263960500737004306F000000A9
:1035300017D70100130787FF83270700638A070057
:10354000737004306F000000737004306F0000006F
:10355000130101FF23248100232611008326070085
:10356000032705009386160017D601002320D6FCFA
:1035700097D60100938686FD83A606003304B70024
:103580002320850063F0E6046372E40263F08602A0
:1035900097D701009387C7FC03A5070013054500D3
:1035A000EFD08FA313050400EF505020EFF0DFD7CA
:1035B000630E05008320C100032481001301010173
:1035C00067800000E366E4FC6FF05FFC0324810089
:1035D0008320C100130101016FC09FFB630E050032
:1035E00017D70100130787F48327070063880700B4
:1035F000737004306F0000006FC09FF9130101FF6A
:1036000023261100232481000327070093070500C8
:103610001307170097D6010023AAE6F097D60100FA
:10362000938606F417D70100130747F20327070014
:1036300003A506003304F70013054500EFD0CF992A
:1036400013050400EF509016EFF01FCE631A05002B
:10365000032481008320C100130101016FC05FF3C7
:103660008320C10003248100130101016780000051
:10367000130101FF232481002326110097D70100A5
:103680009387C7EA83A707001304000093871700F6
:1036900017D70100232CF7E897D70100938747EB52
:1036A00083A7070063EEF51417DE0100130E0E0961
:1036B00097D20100938202FC13040000130700005C
:1036C000930F10001303500A6F00C000130ECEFEBC
:1036D0006384C20F83278EFF93060700E38807FEEB
:1036E0008327CEFF83A74700232EFEFE6386C713E2
:1036F00003AFC70083A747003307E500930E000020
:10370000232EFEFE6380C70983A8C7009387480362
:10371000232017012322F70083A788042326F7011B
:103720002324F70083A7C8022328F70083A70805EE
:10373000232C0700232AF70003A808038347080067
:1037400063986704930708009387170083C60700F0
:10375000B3850741E38A66FE93D52500939505015D
:1037600093D50501231EB700938E1E001307070291
:10377000630A1F038327CEFF83A74700232EFEFE85
:10378000E394C7F983274E00232EFEFE6FF0DFF788
:1037900093050000231EB700938E1E001307070237
:1037A000E31A1FFD3304D40113175400130ECEFE89
:1037B00093060700E390C2F397D70100938707DAD7
:1037C00003AE070083270E006396071297D7010008
:1037D000938787D803AE070083270E00639A071CE0
:1037E00017DE0100130ECEE983274E10639C0702FB
:1037F00083278E11639C072663040600232006009E
:10380000EFF09FB2130504008320C1000324810060
:10381000130101016780000083274E00232EFEFE66
:103820006FF01FED83278E1017DF0100130F0FF6C7
:1038300083A7470017D701002328F7F46386E73DE5
:1038400083A2C70083A74700B306D500930E0000EC
:1038500017D70100232AF7F2930F40001303500AF1
:103860006382E70983A8C7009387480323A0160152
:1038700023A2F60083A7880423A6F60123A4F6005A
:1038800083A7C80223A8F60083A7080523AC060077
:1038900023AAF60003A8080383470800639A673247
:1038A000930708009387170003C70700B3850741F4
:1038B000E30A67FE93D725009397070193D7070183
:1038C000239EF600938E1E0093860602638C1231AF
:1038D00083278E1083A7470017D701002326F7EA16
:1038E000E392E7F983270E1117D70100232EF7E89B
:1038F0006FF05FF783274E00130F8E0083A64700FB
:103900002322DE006380E633B307E50003A7460009
:1039100083A2C600930E00002322EE00930F200026
:103920001303500A6300EF088328C7001387480376
:1039300023A0170123A2E70003A7880423A6F70109
:1039400023A4E70003A7C80223A8E70003A70805EC
:1039500023AC070023AAE70003A8080303470800D5
:10396000631E67221307080013071700834607002A
:10397000B3050741E38A66FE13D725001317070135
:1039800013570701239EE700938E1E0093870702BB
:103990006380122383264E0003A746002322EE00F5
:1039A000E314EFF80327CE002322EE006FF0DFF7D9
:1039B00083274E00130F8E0083A747002322FE00AB
:1039C000638CE72583A2C70083A74700B306D50011
:1039D000930E00002322FE00930F20001303500AD1
:1039E0006300FF0883A8C7009387480323A016013C
:1039F00023A2F60083A7880423A6F60123A4F600D9
:103A000083A7C80223A8F60083A7080523AC0600F5
:103A100023AAF60003A808038347080063986714E5
:103A2000930708009387170003C70700B385074172
:103A3000E30A67FE93D725009397070193D7070101
:103A4000239EF600938E1E0093860602638A12134D
:103A500083274E0083A747002322FE00E314FFF8CC
:103A60008327CE002322FE006FF0DFF78327CE11DD
:103A700097DE0100938ECED283A7470017D70100AF
:103A8000232EF7D0638AD71783AFC70083A74700D9
:103A90003307D5001303000097D6010023A0F6D00A
:103AA000130F3000930220009308500A6388D7094F
:103AB00003A5C700930745032320A7002322F7008F
:103AC000832785042326E7012324F7008327C502E3
:103AD0002328F700832785026384070023265700E5
:103AE00083270505232C0700232AF7000328050355
:103AF00083470800639C1705930708009387170006
:103B000083C60700B3850741E38A16FF93D72500D4
:103B10009397070193D70701231EF70013031300A0
:103B200013070702638EAF028327CE1183A74700D6
:103B300097D6010023A4F6C6E39CD7F783274E123D
:103B400097D6010023ACF6C46FF09FF693070000F0
:103B5000231EF7001303130013070702E396AFFCBD
:103B600033046400E31C06C86FF09FC9930700008C
:103B7000239EF600938E1E0093860602E39A12EDB2
:103B800017DE0100130ECEAF83274E103304D4018D
:103B900093165400E38E07C46FF0DFC813070000CC
:103BA000239EE700938E1E0093870702E39412DFA3
:103BB00097D701009387479A03AE07003304D401D7
:103BC0009316540083270E00E38C07C06FF05FDE6E
:103BD00093070000239EF600938E1E009386060234
:103BE000E39812CF83278E113304D4019316540027
:103BF000E38407C06FF09FE783274E1217D70100B9
:103C0000232EF7B86FF05FE883270E1117D7010056
:103C1000232CF7B66FF0DFC28327CE002322FE00ED
:103C20006FF05FDA8326CE002322DE006FF0DFCD57
:103C3000130101FD2322910223202103232E3101B0
:103C4000232C4101232A51012328610123267101DC
:103C5000232611022324810297D901009389098D1B
:103C600017D901001309C9A117DA0100130A8A8DB7
:103C700097DA0100938ACA8E97DB0100938B4B8DF4
:103C800097D401009384048D130B10006F00000281
:103C900083A70900032449109387170017D7010051
:103CA0002326F788EFF04FE8631E040083A7040083
:103CB000E39007FE83270900E37AFBFEEFC05F8DE8
:103CC0006FF0DFFE7370043083270A00639E0704E1
:103CD0008327091103A4C70013054400EFC0DFAF19
:103CE00083A70B009387F7FF17D701002322F786DE
:103CF00083A704009387F7FF17D70100232CF784CD
:103D000083270A006388070083A70A0083A7470464
:103D10006398070203250403EF200039130504000C
:103D2000EF2080386FF09FF803A70A0083A70A00EE
:103D300083274704938717002322F7046FF05FF966
:103D400003A70A0083A60A00832747049387F7FF87
:103D50002322F70483A74604E39E07FA7360043026
:103D60006FF05FFB97C701009387477C83A707002D
:103D7000639E070E130101FF2326110023248100F7
:103D80002322910097C7010023AA077A17C70100D1
:103D90001307077D83270700B7A6A5A59386565A64
:103DA00083A7070383A50700639ED50003A64700EA
:103DB000631AB60083A687006396C60083A7C70070
:103DC000638AD700032507008325070093854503F1
:103DD000EF30007F17C7010013070777832607001E
:103DE00017D401001304C4896F0000028327070061
:103DF00063860708832707009387F7FF97C60100AC
:103E000023A4F6748326070093972600B387D70070
:103E100093972700B307F40083A70700E38807FC04
:103E20000325070093172500B387A7009397270062
:103E30003307F4008326470093878700B307F40015
:103E400083A4460023229700638EF40283A7C40054
:103E50008320C1000324810017C701002322F770CB
:103E600083244100130101016780000093071000C3
:103E700017C701002324F76C6780000073700430BB
:103E80006F00000083A4440093054001EF508004BC
:103E90003305A400232295006FF05FFB130101FEA0
:103EA00023282101232E1100232C8100232A910095
:103EB00023263101130905007370043097C40100F3
:103EC0009384446883A7040017C401001304446961
:103ED000639C070C6314090003290400930949003B
:103EE00013850900EFC05F8F83278902638607006F
:103EF00013058901EFC05F8E9385090017D5010076
:103F000013058589EFC01F8583A704006388070018
:103F10008327040083A747046394070A83270400C8
:103F20006384270D83A7040063820706737004303F
:103F300083A704006398070E97C701009387076261
:103F400003A70700032707006310070C9307F0FF80
:103F500017C70100232EF75C83A7040063880702BC
:103F60008327040083A74704638207020327040012
:103F700083260400832747049387F7FF2322F7044F
:103F800083A7460463940700736004308320C10153
:103F90000324810183244101032901018329C100F4
:103FA0001301010267800000032704008327040037
:103FB00083274704938717002322F7046FF09FF1AC
:103FC0000327040083260400832747049387F7FF11
:103FD0002322F70483A74604E39207F473600430B6
:103FE00083270400E39027F583A704006382070674
:103FF00097C701009387875383A707006388070A41
:10400000737004306F00000083A7070083A7C70008
:1040100083A7C70083A7470017C70100232AF750CB
:104020006FF09FF3032704008327040083274704CE
:10403000938717002322F70497C70100938707523D
:1040400003A7070003270700E30207F06FF0DFFB79
:1040500097C701009387C74F17C70100130747622F
:1040600083A70700032787116314F7028320C10188
:104070000324810197C7010023A4074E8324410133
:10408000032901018329C100130101026780000097
:10409000032481018320C1018324410103290101FB
:1040A0008329C100130101026FF0DFCB03248101DA
:1040B0008320C10183244101032901018329C10017
:1040C000130101026FC0CFCC6306050A130101FF83
:1040D0002322910097C40100938484482320210166
:1040E0001389050083A504002326110023248100E1
:1040F00093858501EFC00FE903A504001305450072
:10410000EFC08FED9307F0FF630AF90697C7010030
:104110009387C74303A4070003A7040083A70700EE
:104120003304240123228700636EF40697C701003D
:104130009387C74203A5070083A504009385450024
:10414000EFC04FE497C701009387873E83A707001E
:104150006376F40097C7010023AC873C8320C1003D
:10416000032481008324410003290100130101017C
:1041700067800000737004306F00000083A50400A6
:10418000032481008320C10083244100032901000E
:1041900017C5010013054560938545001301010112
:1041A0006FC04FDB97C701009387073B03A507004C
:1041B0000324810083A504008320C10083244100DF
:1041C0000329010093854500130101016FC08FDBB6
:1041D000630E050097C701009387473583A7070043
:1041E000639A0700737004306F000000737004302E
:1041F0006F000000130101FF2322910097C401000A
:104200009384043603A704009387050083A5040064
:10421000B7060080B3E7D7002326110023248100CE
:10422000232CF7009385850113040600EFC08FD27D
:1042300003A5040013054500EFC00FDA9307F0FF54
:104240006304F40297C701009387473003A5070072
:104250008320C100832441003305850003248100AD
:10426000130101016F40905483A5040003248100D1
:104270008320C1008324410017C501001305C551E7
:1042800093854500130101016FC0CFCC6308050A77
:10429000130101FF2322910097C401009384442C51
:1042A000232021011389050083A504002326110082
:1042B000232481009385850113040600EFC08FC974
:1042C00003A5040013054500EFC00FD193071000AC
:1042D000630AF40697C701009387472703A40700E2
:1042E00003A7040083A707003304240123228700C7
:1042F000636EF40697C701009387472603A507005E
:1043000083A5040093854500EFC0CFC797C7010080
:104310009387072283A707006376F40097C70100FD
:1043200023A887208320C100032481008324410027
:10433000032901001301010167800000737004303C
:104340006F00000083A50400032481008320C100C6
:10435000832441000329010017C501001305C5434B
:1043600093854500130101016FC0CFBE97C70100BF
:104370009387871E03A507000324810083A50400FB
:104380008320C10083244100032901009385450057
:10439000130101016FC00FBF130101FF232611009C
:1043A00023248100232291008327C50003A4C70092
:1043B0006304040A9304840113850400EFC0CFC191
:1043C00097C701009387871683A70700639A07089A
:1043D0009304440013850400EFC00FC097C7010089
:1043E000938787160327C40283A7070063F6E700B5
:1043F00097C7010023AAE71493172700B387E700A4
:104400009397270017C5010013058527938504009E
:104410003305F500EFC00FB497C701009387471429
:1044200083A707000327C4021305000083A7C70260
:1044300063FAE7009307100017C701002320F71065
:10444000130510008320C100032481008324410050
:104450001301010167800000737004306F000000D9
:104460009385040017C5010013058530EFC08FAE9A
:104470006FF09FFA97C701009387470B83A7070048
:1044800063960700737004306F000000130101FF92
:10449000232611002324810023229100B7070080E6
:1044A0000324C500B3E7F5002320F50063080408E2
:1044B000EFC08FB29304440013850400EFC0CFB166
:1044C00097C70100938747080327C40283A7070003
:1044D00063F6E70097C7010023A8E70693172700B4
:1044E000B387E7009397270017C501001305451907
:1044F0003305F50093850400EFC0CFA597C70100F1
:104500009387070683A707000327C402130500004B
:1045100083A7C70263FAE7009307100017C70100DB
:10452000232EF700130510008320C100032481000F
:10453000832441001301010167800000737004307F
:104540006F0000006304050297C701009387C7FE50
:1045500003A7070097C70100938747FF83A70700BA
:104560002320E5002322F5006780000073700430EB
:104570006F0000006304050E638E050C130101FF3C
:1045800023261100232481001307050073700430D3
:1045900097C80100938808FB83A70800638007027F
:1045A00097C701009387C7FB83A6070083A707006F
:1045B00083A746049387170023A2F60417C30100BC
:1045C0001303C3F883A70500032603009306F0FF37
:1045D000130400006388D70417CE0100130ECEF534
:1045E00003250E0003280700832647006306A80062
:1045F000130410006378D6023308D6401304100069
:104600006372F80203250E00B387C7400326030038
:10461000B387D70023A0F5002320A7002322C700DB
:104620001304000083A70800638C070097C70100EC
:10463000938707F383A7070083A7470463940702C0
:10464000130504008320C10003248100130101012C
:1046500067800000737004306F00000073700430D6
:104660006F000000EF40101D6FF09FFD93071000DA
:1046700017C701002324F7EC6780000063060500DC
:104680000325C50467800000130500006780000053
:10469000630405002326B5046780000097C7010066
:1046A000938707EC03A507006780000097C7010008
:1046B000938747E983A7070013051000638C070061
:1046C00097C70100938787E603A5070013351500F8
:1046D0001315150067800000630C0508130101FE27
:1046E000232A910097C40100938484E783A70400E0
:1046F000232E1100232C81002328210123263101A0
:104700000327C50283A7C7026376F70483278501C1
:1047100063CC070083A7040083A6C7029307A00009
:10472000B387D740232CF50093172700B387E70002
:104730000327450117C90100130989F4939727003E
:10474000B307F9006308F70283A7040083A7C70231
:104750002326F5028320C101032481018324410122
:10476000032901018329C1001301010267800000B0
:1047700067800000930945001304050013850900B4
:10478000EFC08F8583A7040017C701001307C7DB9D
:104790000327070083A7C7022326F4026376F700E6
:1047A00017C701002322F7DA139527003305F50018
:1047B00003248101131525008320C10183244101B5
:1047C000938509003305A9008329C100032901014C
:1047D000130101026FB01FF863060502130101FF08
:1047E00023261100232481002322910097C7010072
:1047F000938707D703A40700630AA40073700430EB
:104800006F00000013050000678000008327440547
:1048100063960700737004306F0000008326C402A3
:10482000032704059387F7FF232AF4046384E60033
:10483000638E0700130500008320C100032481005C
:1048400083244100130101016780000093044400A8
:1048500013850400EFB05FF80325040597C7010036
:10486000938787CE03A707009307A000B387A740CD
:104870002326A402232CF4006376A70097C7010027
:1048800023A4A7CC93054001EF40C06497C7010063
:10489000938707DF3385A70093850400EFB09FEB74
:1048A000130510006FF05FF97370043097C70100B3
:1048B000938747C983A707006380070297C7010052
:1048C000938707CA03A7070083A707008327470426
:1048D000938717002322F7046780000097C7010021
:1048E000938747C683A70700638C070297C7010019
:1048F000938707C703A7070003274704630207023C
:1049000003A7070083A60700832747049387F7FFC1
:104910002322F70483A746046394070073600430DE
:104920006780000097C70100938787C303A607002D
:1049300083A6070003A707009307A00083A6C6026B
:1049400003258601B387D740232CF700678000003A
:1049500097C701009387C7C003A70700630A070032
:1049600083A6070003A746051307170023AAE6043A
:1049700003A5070067800000130101FD2320210328
:10498000232611022324810223229102232E3101A6
:10499000130905007370043097C40100938484BA2E
:1049A00083A7040017C40100130484BB639E070A95
:1049B0008327040083A78705639A070083270400E1
:1049C0001307100023AEE704639A050E83A70400C3
:1049D000638807008327040083A74704639A0714AA
:1049E0007370043083A704006394070683270400D0
:1049F00003A58705630805006302090483270400F3
:104A000023AC07048327040023AE070483A7040014
:104A1000638807008327040083A74704639207067F
:104A20008320C1020324810283244102032901025D
:104A30008329C101130101036780000003270400DB
:104A4000832787059387F7FF232CF7046FF09FFBDD
:104A50000327040083270400832747049387170054
:104A60002322F7046FF09FF8032704008327040034
:104A700083274704938717002322F7046FF05FF31F
:104A80000327040083260400832747049387F7FF46
:104A90002322F70483A74604E39407F873600430E5
:104AA0008320C102032481028324410203290102DD
:104AB0008329C1011301010367800000032504005D
:104AC0002326B10013054500EFB01FD18325C10097
:104AD0009307F0FF6380F50897C70100938707A746
:104AE00083A907000327040083A70700B389B9003F
:104AF0002322370163ECF90697C70100938707A6C5
:104B000003A507008325040093854500EFB09FC7E8
:104B100097C701009387C7A183A7070063F6F90031
:104B200097C7010023A637A1EFB09FA66FF01FEA39
:104B30000327040083260400832747049387F7FF95
:104B40002322F70483A74604E39C07E8736004303C
:104B50006FF01FE98325040017C501001305C5C3C5
:104B600093854500EFB01FBF6FF01FFC97C7010092
:104B70009387879E03A5070083250400938545003E
:104B8000EFB05FC06FF05FFA130101FD2320210336
:104B9000232E310123261102232481022322910294
:104BA000232C41011389050093090600737004301A
:104BB00097C401009384049983A7040017C40100DB
:104BC0001304049A639C071403270400930720002E
:104BD0000327C7056304F702832704001345F5FF85
:104BE00003A787053375E50023ACA70483270400DA
:104BF0001307100023AEE704639A060A83A7040094
:104C0000638807008327040083A74704639407167B
:104C10007370043083A70400639E0706638809004D
:104C20008327040083A7870523A0F9000327040036
:104C300093071000130500000327C705630EF70054
:104C4000832704001349F9FF1305100003A7870504
:104C50003379E90023AC27058327040023AE07043A
:104C600083A70400638807008327040083A7470401
:104C70006392070C8320C102032481028324410232
:104C8000032901028329C101032A810113010103C0
:104C9000678000000327040083270400832747045C
:104CA000938717002322F7046FF05FF703250400B2
:104CB0002326D10013054500EFB01FB28326C100A3
:104CC0009307F0FF638AF60C97C701009387078864
:104CD00003AA07000327040083A70700330ADA00AA
:104CE000232247016368FA0C97C70100938707875F
:104CF00003A507008325040093854500EFB09FA816
:104D000097C701009387C78283A707006370FA0AD9
:104D100097C7010023AE47816F00400903270400B5
:104D20008327040083274704938717002322F7046F
:104D30006FF09FE9032704008326040083274704BC
:104D40009387F7FF2322F70483A74604E39407F22F
:104D5000736004308320C102032481028324410252
:104D6000032901028329C101032A810113010103DF
:104D7000678000000327040083260400832747047C
:104D80009387F7FF2322F70483A74604E39207E8FB
:104D9000736004306FF0DFE78325040017C501005E
:104DA0001305859F93854500EFB0DF9AEFB04FFE66
:104DB0006FF0DFE497B701009387077A03A5070038
:104DC0008325040093854500EFB0DF9B6FF01FFE45
:104DD000630A050C130101FF23261100232481001F
:104DE00023229100232021017370043097B4010025
:104DF0009384447583A704006396070863860600BE
:104E00008327850523A0F60093070600930620005C
:104E10000326C505232ED5041387050013040500BA
:104E20006382D70A63F4F608930530006388B700FD
:104E3000930540006396B700630CD610232CE4045E
:104E400093071000630CF6081304100083A70400F6
:104E5000638C070097B701009387877083A70700CB
:104E600083A7470463980706130504008320C10045
:104E7000032481008324410003290100130101015F
:104E80006780000097B701009387876D03A707002D
:104E900083A7070083274704938717002322F7047B
:104EA0006FF0DFF5737004306F00000093061000A0
:104EB000E398D7F88327850533E7B700232CE5046B
:104EC0006FF01FF88327850593871700232CF504BF
:104ED0006FF01FF7EF4000166FF01FF91309440041
:104EE00013050900EFB05F8F97B701009387C7657F
:104EF0000325C40283A7070063F6A70097B7010044
:104F000023A4A76493054001EF30D07C97B701003C
:104F1000938707773385A70093050900EFB09F8338
:104F20008327840263860700737004306F000000DB
:104F300097B701009387C76283A707000327C402BE
:104F400083A7C702E3F2E7F0EFB08FE46FF0DFEF83
:104F5000130400006FF09FEF63080508130101FEC2
:104F6000232C8100232A91002328210123263101AB
:104F70002324410123225101232E1100930907000C
:104F8000138A060093040600138905001304050024
:104F9000EFB04FF4930A050063060A0083278405E7
:104FA0002320FA000327C40593072000232EF404CE
:104FB0006380F40463FA9710930630006388D4008A
:104FC000930640006396D400630CF70E232C24054F
:104FD000930710006312F70A832784026382070293
:104FE000737004306F000000737004306F000000B5
:104FF0008327840593871700232CF4046FF05FFD4B
:1050000097B701009387875283A707006390070A29
:105010009304440013850400EFB00FFC97B7010020
:10502000938787520325C40283A7070063F6A7006E
:1050300097B7010023AAA75093054001EF3090696C
:1050400097B701009387C763938504003385A70052
:10505000EFB04FF097B701009387875083A7070001
:105060000327C40283A7C70263F8E7006386090029
:105070009307100023A0F9001304100013850A0001
:10508000EFB0CFE4130504008320C10103248101A4
:1050900083244101032901018329C100032A8100DE
:1050A000832A4100130101026780000093058401F7
:1050B00017B501001305C56BEFB0CFE96FF09FF98D
:1050C000130400006FF09FFB93071000E392F4F0CD
:1050D0008327840533E92701232C24056FF05FEF34
:1050E000630A050E130101FE232C8100232A91007F
:1050F0001304050023263101232E1100232821014A
:1051000093840500EFB00FDD930720008326C405CC
:10511000232EF40483278405130710009309050048
:1051200093871700232CF4046396E60883278402F0
:1051300063860700737004306F00000097B70100AA
:105140009387C73E83A70700639A070813094400A3
:1051500013050900EFB04FE897B701009387C73EEA
:105160000325C40283A7070063F6A70097B70100D1
:1051700023ACA73C93054001EF30D05597B7010011
:1051800093870750930509003385A700EFB08FDCA4
:1051900097B701009387C73C83A707000327C40282
:1051A00083A7C70263F8E700638604009307100033
:1051B00023A0F400032481018320C1018324410141
:1051C00003290101138509008329C100130101028C
:1051D0006FB0CFCF737004306F000000930584016F
:1051E00017B501001305C558EFB0CFD66FF05FFAC1
:1051F00093070500630805067370043017B70100B4
:105200001307473483260700639E060203A6C705DB
:1052100093062000130500006316D60023AE070492
:105220001305100083270700638C070097B7010060
:105230009387073303A7070003274704631C07026C
:105240006780000097B601009386863103A60600AA
:1052500083A6060083264604938616002322D604DE
:105260006FF0DFFA97B701009387872F83A70700B6
:105270006FF09FF803A7070083A607008327470462
:105280009387F7FF2322F70483A74604E39A07FADC
:105290007360043067800000130101FB2322910436
:1052A00023202105232C4103232A510323286103B2
:1052B000232671032326110423248104232E310382
:1052C00023248103232291032320A10317B9010082
:1052D0001309092A17BB0100130BCB2897B401004F
:1052E0009384842897BA0100938A4A28130A1000ED
:1052F000930B90008327090003A707006306071696
:1053000083A7C70083A90700EFD09FCEEFD0DFCFE0
:1053100083270B00130C05006368F50C97B7010099
:1053200023A2A724130600006376352303A50400F7
:10533000B3858941EFC09F9EEFD01FFF630605161E
:1053400003A50400930600001306000093058100E6
:10535000EFC08FADE30005FA83278100E3C207FEAB
:105360008329010183A7490163860700138549004A
:10537000EFB08FC6EFD05FC983270B00130C050079
:105380006362F50C8327810017B70100232C871D6A
:10539000E3E8FBFAB317FA0013F7072163100720BD
:1053A00013F7770C6316072A93F70702E38A07F8C7
:1053B00013850900EF00504F6FF09FF883A7C700D7
:1053C00003A4C70083AC07009309440013850900B8
:1053D000EFB08FC08327440213050400E780070065
:1053E0008327C4016386470D8327090003A70700AD
:1053F000E31607FC03A70A0097B6010023A486174B
:1054000097B6010023A4F61697B7010023A2E7166A
:10541000EFD09FF16FF0DFF283A7C70003A4C700AE
:1054200003AD0700930C440013850C00EFB0CFBA16
:105430008327440213050400E78007008327C40183
:10544000638C470B8327090003A70700E31607FCBB
:1054500003A70A0097B6010023AAF61097B7010028
:1054600023A8E7106FF01FF2EFD09FB8EFD0DFB99D
:1054700083270B00130C0500E368F5F683A70A00E9
:1054800003A504009309000003A60700B385894122
:1054900017B701002328870D13361600EFC01F88A9
:1054A000EFD09FE8E31E05E8EFB08F8E6FF05FE965
:1054B0008327840193850900B387FC0063E2FC081D
:1054C00083A7040063860702232A0100232C91018D
:1054D000232E8100EFF08F9D03A5040093060000AA
:1054E0001306000093054101EFB0DFACE31E05EEAB
:1054F000737004306F0000008327840193850C00D3
:10550000B307FD006362FD0883A7040063860702FA
:10551000232A0100232CA101232E8100EFF00F99F3
:1055200003A5040093060000130600009305410143
:10553000EFB05FA8E31805F0737004306F0000004F
:10554000032509002322F40023288400EFB08FA351
:105550006FF09FE9EFD05FDD8327090083A7C700C5
:1055600003A4C700930C440013850C00EFB0CFA632
:105570008327C401638A4705832744021305040077
:10558000E78007006FF0DFDB032509002322F4002A
:1055900023288400EFB00F9F6FF0DFEA8327C1005C
:1055A00023ACF9006382070AB387870123A2F900BD
:1055B00023A83901938549006362FC0803A50A000A
:1055C000EFB04F9C6FF0DFD783278401232884003E
:1055D0003387F9002322E400636AEC04330C3C4176
:1055E000636EFC0283A7040063860702232A01007E
:1055F000232C3101232E8100EFF04F8B03A50400F3
:10560000930600001306000093054101EFB09F9A36
:10561000E31405F6737004306F00000003A50A0060
:1056200093850C00EFB00F966FF01FF5032509006E
:1056300093850C00EFB00F956FF01FF40325090060
:10564000EFB04F946FF0DFCF737004306F00000045
:105650008327C10083A6890123A839013387D70096
:1056600023A2E9006362EC06B307FC4063EAD706B5
:1056700083A7490213850900E780070083A7C901B2
:10568000E39047CD83A689018327C10003A70400C7
:10569000B387D70063060702232A0100232CF100F9
:1056A000232E3101EFF08F8003A504009306000044
:1056B0001306000093054101EFB0DF8FE31205C828
:1056C000737004306F0000006374FC00E372F7FA3B
:1056D0000325090093854900EFB0CF8A6FF05FC6BC
:1056E00003A50A0093854900EFB0CF896FF05FC52D
:1056F000130101FF2324810023261100232291009E
:105700002320210117B40100130404E6EFF0CF9920
:105710008327040063840704EFF04F9C8327040071
:10572000638A070293080000130800009307000033
:1057300013072000930600001306004097B50100F0
:105740009385C5C717050000130545B5EFC01F9E1B
:1057500063140506737004306F00000017B9010070
:105760001309C90413050900EFA05FFC97B40100F9
:105770009384040513850400EFA05FFB130600006B
:105780009305C0001305400097B7010023A227DF4F
:1057900097B7010023AC97DCEFB08FC817B70100B3
:1057A0002324A7DC6306050297B50100938585C015
:1057B000EFC08FC36FF05FF68320C1000324810028
:1057C00083244100032901001301010167800000C7
:1057D000737004306F000000638A050A130101FD35
:1057E000232A5101930A05001305C00223248102D4
:1057F0002322910223202103232E3101232C410156
:1058000023261102232861012326710113090700B1
:1058100093890600130A060093840500EF00C07008
:1058200013040500630C0502EFF00F8897B7010021
:10583000938787D383A70700638E0704EFF00F8A4F
:105840001305440023205401232C9400232E4401EB
:105850002320340323222403EFA05FEF1305040069
:105860008320C1020324810283244102032901020F
:105870008329C101032A8101832A4101032B0101EC
:10588000832BC10013010103678000007370043093
:105890006F00000097BB0100938B4BF113850B0049
:1058A000EFA0DFE817BB0100130B8BF113050B0012
:1058B000EFA0DFE7130600009305C00013054000CA
:1058C00097B7010023A677CB97B7010023A067CB3A
:1058D000EFB00FB517B701002328A7C8630A05006A
:1058E00097B50100938505ADEFC00FB06FF01FF5C0
:1058F000737004306F000000630E0506130101FE93
:10590000232C8100232E1100232A910017B40100BB
:10591000130484C583280400130805001305000040
:1059200063800804930407002322B1001387060054
:105930002324C100232601019306500063C0B6044E
:10594000EFE0DFD693072000630EF5040325040083
:10595000930600001306000093054100EFB08FE5A9
:105960008320C10103248101832441011301010229
:1059700067800000737004306F00000093054100E1
:10598000930600001306070013850800EFB05F9828
:105990008320C101032481018324410113010102F9
:1059A00067800000032504009306000013860400AE
:1059B00093054100EFB00FE06FF09FFA630605001A
:1059C0000325050067800000737004306F0000003D
:1059D00063160500737004306F000000130101FFAF
:1059E000232611002324810013040500EFE0DFEBE0
:1059F000032544013334A000EFE05FEE13050400FB
:105A00008320C1000324810013010101678000008D
:105A100063160500737004306F000000130101FF6E
:105A2000232481001304050023261100EFE0DFE7A3
:105A300003240402EFE09FEA8320C1001305040061
:105A40000324810013010101678000006316050033
:105A5000737004306F000000130101FF23248100E4
:105A600023229100138405009304050023261100CE
:105A7000EFE09FE323A08402032481008320C10080
:105A800083244100130101016FE05FE5130101FF71
:105A90001305C0012324810023261100EF00C04814
:105AA00013040500630805002320050013054500C5
:105AB000EFA0DFC7130504008320C1000324810089
:105AC000130101016780000063020502B70700FFB0
:105AD000B3F7F50063860700737004306F000000B1
:105AE000639A0500737004306F0000007370043017
:105AF0006F000000130101FE232C810023282101E7
:105B0000232631012324410123225101232E110098
:105B1000232A91009309070013890600930A0600BF
:105B200013840500130A0500EFE05FB86318050051
:105B300063860900737004306F000000EFD04FCB14
:105B400083240A00B3779400631209046382070474
:105B500063880A009347F4FFB3F797002320FA0005
:105B6000EFD08FFC8320C101032481011385040041
:105B700003290101832441018329C100032A8100F3
:105B8000832A41001301010267800000E302F4FC54
:105B9000E38809FCB335500193958501630609003C
:105BA000B7070004B3E5F50013860900B3E58500E7
:105BB00013054A00EFE0CFE1EFD00FF763140500C3
:105BC000EFA01F9DEFE01FD6931765009309050016
:105BD00063DA0700B70400019384F4FFB3F499007B
:105BE0006FF05FF8EFE05FCC83290A00B3773401F0
:105BF00063100902638A070063880A009347F4FF71
:105C0000B3F737012320FA00EFE05FCD6FF09FFC80
:105C1000E31CF4FE6FF05FFE630C0500B70700FFA6
:105C2000B3F7F500638A0700737004306F0000005B
:105C3000737004306F000000130101FF2324810002
:105C400013040500232611002322910023202101A3
:105C500013890500EFE05FC5832404009345F9FF35
:105C6000B3F795002320F400EFE05FC78320C10065
:105C700003248100138504000329010083244100CB
:105C80001301010167800000130101FF232481003B
:105C90001304050023261100EFA0DFA30324040052
:105CA000EFA0DFA28320C1001305040003248100BC
:105CB0001301010167800000630C0500370700FF36
:105CC000B3F7E500638A0700737004306F000000CB
:105CD000737004306F0000006F308038B70700FF2A
:105CE000B377F60063860700737004306F0000001E
:105CF00063160600737004306F000000130101FE8C
:105D0000232C810023282101232631012324410152
:105D1000232E1100232A9100138906009389050080
:105D2000130A050013040600EFE05F98631E0504E4
:105D300063060900737004306F000000EFD04FABB2
:105D400083240A009385090013050A00B3E499002F
:105D5000EFF09FF6B3779400630AF40883240A00F7
:105D6000EFD08FDC8320C10103248101138504005F
:105D700003290101832441018329C100032A8100F1
:105D80001301010267800000EFD08FA683240A0070
:105D90009385090013050A00B3E43401EFF0DFF145
:105DA000B3F7840063848704E30A09FAB7050005A2
:105DB00013060900B365B40013054A00EFE04FC1B4
:105DC000EFD08FD663140500EFA08FFCEFE09FB5F6
:105DD000931765009304050063D40702B707000119
:105DE0009387F7FFB3F4F4006FF0DFF783270A001F
:105DF0001344F4FFB3F787002320FA006FF05FF637
:105E0000EFE09FAA83240A00B37794006398870089
:105E10009347F4FFB3F797002320FA00EFE01FAC9D
:105E20006FF0DFFB130101FF232481002326110003
:105E30001304050023229100EFD08F9B8327440099
:105E400063860702032504019304C40063189500C8
:105E50006F0080030325040163089502B705000263
:105E6000EFE04FE183274400E39607FE13050400AB
:105E7000EF008023032481008320C100832441009C
:105E8000130101016FD04FCA737004306F0000001E
:105E9000630C0500370700FFB3F7E500638A0700CE
:105EA000737004306F000000737004306F000000E6
:105EB0006F30001B630C0500B70700FFB3F7F50058
:105EC000638A0700737004306F0000007370043041
:105ED0006F000000130101FF2324810023229100A1
:105EE000232611001304050093840500EFE0DF9BD7
:105EF0000327040093C7F4FFB377F7002320F400CF
:105F0000032481008320C100832441001301010187
:105F10006FE0DF9C630605000325850167800000B4
:105F20001305000067800000130101FF2324810096
:105F30002326110013040500EFD08F8B97A70100D3
:105F40009387476383A70700639C0704B797010003
:105F500017B70100130747889387C7FF97A601006B
:105F600023A0E66217A70100232AF76017B70100F4
:105F70002326F78697A701009387076017B70100CC
:105F8000232CF7849307100017A70100232C075E2A
:105F900017A701002322075E17A70100232CF75C37
:105FA00063120402EFD04FB8EF10C060130400007A
:105FB000130504008320C1000324810013010101A3
:105FC0006780000013058400937735006398070C01
:105FD000B79701001307F5FF9387A7FFE3E4E7FCFA
:105FE00097A601009386C65983A706006F0040015B
:105FF00003A70700630A07009386070093070700BB
:1060000003A74700E366A7FE17A701001307C756BB
:10601000E38AE7F803A7070013060001138487004B
:1060200023A0E60003A74700B306A740637ED6027D
:106030003388A7002322D80023A2A7008325480085
:1060400097A601009386C6536F0080009306070051
:1060500003A7060003264700E36AB6FE2320E800F4
:1060600023A0060103A7470097A701009387475580
:1060700083A70700B387E74017A701002322F7543F
:10608000EFD08FAAE30204F2130504008320C100BD
:106090000324810013010101678000001375C5FF0F
:1060A000130545006FF0DFF263080506130101FFD9
:1060B000232481002326110013040500EFC05FF3A1
:1060C000930584FF0326C4FF17A701001307474B5E
:1060D0006F008000138707008327070083A647000F
:1060E000E3EAC6FE232CF4FE2320B70097A70100A5
:1060F0009387074D03A707008327C4FF032481006C
:106100008320C100B387E70017A70100232AF74ABD
:10611000130101016FD04FA16780000097A7010014
:106120009387074A03A50700678000006780000087
:106130003367B50013773700930705006312070430
:106140009308D6FFB30815011307050093860500D1
:106150006378150303A806001307470093864600DB
:10616000232E07FFE36817FF9347F5FFB387170157
:1061700093F7C7FF93874700B385F500B307F50092
:106180003306C50063F4C70C9386450013884700A7
:10619000B3B6D70033B8050133E7F50093C6160050
:1061A0001348180013773700B3E6060113371700BA
:1061B0003377D700330EF64093861700630807063F
:1061C0001337AE006314070613532E00138805001F
:1061D00093860700130700008328080013071700A1
:1061E0001308480023A0160193864600E36667FE65
:1061F0001377CEFFB385E500B387E7006306EE04AF
:1062000083C60500138717002380D700637EC7026B
:1062100083C6150013872700A380D7006376C702C3
:1062200003C725002381E70067800000B307F6401D
:10623000B387F5009385150003C7F5FF9386160015
:10624000238FE6FEE398F5FE67800000678000007C
:10625000B367C50093F73700B308C5006382070E24
:1062600063761511B307A04093F737001387370003
:106270009306500093F5F50F130815003383A840DB
:106280001306F6FF6374D700130750006368E60E29
:106290006380070E2300B50013071000638EE7002C
:1062A000A300B50013073000130825006396E7002C
:1062B000130835002301B5001396850033E6C500A9
:1062C000139705013367E6003303F3409396850186
:1062D000B366D70013562300B307F5001307000079
:1062E00023A0D7001307170093874700E36AC7FE70
:1062F0001377C3FFB307E8006300E3082380B70008
:1063000013871700637C1703A380B7001387270048
:10631000637617032381B700138737006370170371
:10632000A381B70013874700637A17012382B70060
:106330001387570063741701A382B70067800000BA
:1063400093F5F50F13978500B365B7001397050113
:106350003367B700E37415FF930705009387470081
:1063600023AEE7FEE3EC17FF6780000067800000C4
:10637000130805006FF05FF46780000093070500C5
:106380006FF0DFF78347050013070500638C0700F4
:106390001305150083470500E39C07FE3305E54020
:1063A00067800000130500006780000013051500DA
:1063B0008347F5FF9385150003C7F5FF6388070042
:1063C000E386E7FE3385E74067800000930700001F
:1063D0006FF05FFF930705009385150003C7F5FF76
:1063E00093871700A38FE7FEE31807FE678000007E
:1063F00083460500930700026398F6001305150015
:1064000083460500E38CF6FE938756FD93F7D70F7E
:106410006380070493070500930500006388060462
:106420001305000093871700138606FD1317250038
:1064300083C607003305A700131515003305A60012
:10644000E39206FE638405003305A04067800000E8
:10645000938536FD8346150093B515009307150007
:10646000E39006FC130500006FF0DFFD130500004C
:106470006780000083A705002380A70083A705008D
:106480009387170023A0F5006780000097A60100FE
:106490009386860F83A706001737030013078736F6
:1064A00013861700B307F7002380A70097A5010004
:1064B00023ACC50C9307A000630AF5009307000402
:1064C0006308F6001305000067800000E30C06FE79
:1064D000370610F0130717008347F7FF2320F6F065
:1064E00083A706009387F7FF97A5010023AEF50861
:1064F000E39207FE1305000067800000130101EB23
:106500002322911423202115232A5113232481139C
:106510002326111423248114232E3113232C4113F9
:106520002328611323267113232291132320A113FF
:10653000232EB11193040500138905002326C10001
:10654000130C5002930A9000834709006388870365
:10655000638C070603A404006F00800063860706AF
:106560002300F40003A40400130919001304140009
:1065700023A0840083470900E39287FF03461900A4
:106580009308190093860800130D00029309F0FF89
:10659000130AF0FF13080000130550059307D6FDFA
:1065A00093F7F70F13891600636EF53A17A70100EA
:1065B000130747A593972700B387E70083A7070032
:1065C000B387E700678007008320C1140324811488
:1065D00083244114032901148329C113032A81133D
:1065E000832A4113032B0113832BC112032C811225
:1065F000832C4112032D0112832DC11113010115AA
:1066000067800000930C8000232401009307100092
:1066100063DA071D8327C10003A40400938B77006E
:1066200093F68BFF03AB060083A946009387860091
:106630002326F10013860C009306000013050B00BF
:1066400093850900EF2000392328A100930700005B
:1066500063803733930D4101930B100013860C00B8
:106660009306000013050B0093850900EF10D05826
:106670009306000013860C00130B05009389050098
:10668000EF2040358327810023A0AD0093861B00B7
:10669000938D4D0063863701938B06006FF01FFCCE
:1066A000E37C9BFF63D24603930704002380A7018A
:1066B00003A40400130AFAFF9307140023A0F400B4
:1066C00013840700E3C446FF93962B009307010150
:1066D000B386D7006F008002938777052300F4000C
:1066E00003A40400938BFBFF93871B001304140087
:1066F00023A084009386C6FFE358F0E483A7060036
:10670000E3ECFAFC938707036FF05FFD83A70400B7
:10671000930600030327C1002380D70083A704004A
:1067200093064700930C00011386170023A0C400B2
:1067300013068007A380C70003A4040023240100DC
:10674000930707001304140023A0840003AB070081
:10675000930900002326D1006FF0DFED8327C100ED
:1067600083AC0700938B470063880C28635C40254B
:106770009307D002631EFD2083C70C0063880702C5
:1067800063D8092483A60400938C1C00130AFAFF23
:106790002380F60003A404001304140023A0840043
:1067A00083C70C00E39E07FC6352400303A404006C
:1067B000930700022300F40003A40400130AFAFF65
:1067C0001304140023A08400E3160AFE232671019B
:1067D0006FF09FD72324010093071000930CA000B3
:1067E000E3CA07E38327C10003A40400938647009C
:1067F0006FF0DFF503C61600930609006FF01FDA8D
:1068000083A70400930650022380D70003A404004A
:106810001304140023A084006FF01FD3930C000115
:10682000232401006FF09FDE8327C10003C61600FA
:106830009306090083A90700938747002326F100E8
:10684000E35E0AD4138A09009309F0FF6FF01FD5A5
:1068500003C61600130DD002930609006FF01FD473
:106860009347FAFF93D7F74103C61600337AFA002D
:10687000930609006FF09FD203C61600130D0003A4
:10688000930609006FF09FD183C51600930906FD9A
:1068900093060900938705FD13860500E3E2FAFAE3
:1068A00093972900B38937019386160093991900AD
:1068B000B389B90083C50600938909FD938705FD57
:1068C00013860500E3FEFAFC6FF09FF70327C10073
:1068D00083A7040083260700130747002326E1004F
:1068E0002380D70003A404001304140023A0840011
:1068F0006FF09FC59307100063D4070F8327C10073
:106900009386770093F686FF938786002326F1000F
:1069100083A9460083A7060063DE090E83A6040050
:106920001306D002B307F0402380C60003A404007E
:10693000B336F000B30930411304140023A08400DF
:10694000138B0700B389D940930CA00023240100C6
:106950006FF05FCE03C616001308180093060900F7
:106960006FF0DFC383A70400138908006FF09FE96D
:10697000E3729BCF93071000930B00009306100067
:10698000E3C447D36FF05FD497AC0100938C8CA322
:106990009385090013850C00EF10404E330AAA407E
:1069A0006352400303A404002300A40103A40400D1
:1069B000130AFAFF1304140023A08400E3160AFE4E
:1069C000130A000083C70C00E38207E0E3CC09DA76
:1069D0009389F9FF1307F0FFE396E9DA6FF0DFDC44
:1069E0008327C1009386470083A707002326D10091
:1069F00093D9F7416FF05FF2635640019307D002DD
:106A0000E314FDF897AC0100938CCC9B93078002B4
:106A10006FF01FD7138B0700930CA00023240100F5
:106A200003A404006FF01FC1130101EB232E3113E7
:106A3000B70900409387F9FF23248114232291147E
:106A4000232C4113232A511323261114232021150B
:106A500023286113232671132324811323229113E6
:106A60002320A113232EB111130A05002324B10002
:106A700017A40100130444B1973A0300938A8AD8FB
:106A8000979401009384846D2326F10093055002AE
:106A90001305A00013080004B70610F083470A008E
:106AA000638EB7046388070A03270400130A1A00D9
:106AB000130617003387EA0097A8010023A6C8AC85
:106AC0002300F7006380A708E31A06FD17370300C9
:106AD000130747D3130717008347F7FF23A0F6F0E8
:106AE000832704009387F7FF17A60100232EF6A83B
:106AF000E39207FE83470A00E396B7FA83461A003B
:106B000013051A0013070500930B0002130BF0FF87
:106B1000130CF0FF13080000930550059308900034
:106B20009387D6FD93F7F70F130A170063ECF5442C
:106B300093972700B387970083A70700B387970031
:106B400067800700173703001307C7CBE31406F865
:106B50006FF0DFF48320C1140324811483244114D3
:106B6000032901148329C113032A8113832A4113A2
:106B7000032B0113832BC112032C8112832C41128E
:106B8000032D0112832DC11113010115678000002F
:106B9000930C8000130D00009307100063DA0721A7
:106BA000832781009387770093F787FF83AD0700E2
:106BB00003AB4700138787002324E10013860C00F2
:106BC0009306000013850D0093050B00EF109060F5
:106BD0002328A10063086D451309410193091000A2
:106BE00013860C009306000013850D0093050B001F
:106BF000EF10900013860C0093060000930D050023
:106C0000138B0500EF10105D2320A9009389190054
:106C100013094900E3166DFDE3F49DFD130600041E
:106C2000B70610F063D48903832704001387170085
:106C3000B387FA0097A5010023A8E5942380770184
:106C4000630AC706130CFCFFE3C089FF8327C1005A
:106C50001305C10093089000B386F90093962600AF
:106C600093070101B386D7001308A00013030004A3
:106C7000370610F0E38CA6E083A706009305000317
:106C800063F4F8009305700503270400B387B70089
:106C9000930517003387EA0017AE01002326BE8E46
:106CA0002300F70063860737638C65329386C6FF3F
:106CB0006FF05FFC173703001307C7B41307170003
:106CC0008347F7FF23A0F6F0832704009387F7FF9D
:106CD00097A5010023AAF58AE39207FE130CFCFF97
:106CE0006FF09FF683270400130600041387170034
:106CF00097A5010023AAE588B386FA00930500034F
:106D00002380B6006308C7509387270097A6010029
:106D100023ACF6863387EA00930680072300D7006A
:106D200017370300130707AEB70610F06392C702C8
:106D3000130717008347F7FF23A0F6F0832704000B
:106D40009387F7FF17A601002320F684E39207FE3E
:106D500083278100930C0001130D000093874700E7
:106D600003278100130B0000832D07002324F1006B
:106D70006FF0DFE48327810083AC070013894700AD
:106D8000638E0C4C6358802B9307D0026394FB3EB8
:106D900003C70C00930507006314072A6F00002F38
:106DA00093071000930CA000130D0000E3CA07DF47
:106DB00083278100938747006FF09FFA8327810024
:106DC0008346170013070A0003AB070093874700A9
:106DD0002324F100E3560CD4130C0B00130BF0FF2B
:106DE0006FF01FD483461700930BD00213070A00DD
:106DF0006FF01FD39347FCFF93D7F74183461700EB
:106E0000337CFC0013070A006FF09FD18346170004
:106E1000930B000313070A006FF09FD0034617007F
:106E2000138B06FD13070A00930706FD9306060061
:106E3000E3E2F8FA93172B00B387670113071700F3
:106E400093971700B387C70003460700138B07FD0E
:106E5000930706FD93060600E3FEF8FC6FF09FF72C
:106E600083258100832704001306A00003A70500E3
:106E700093861700B387FA00179501002326D57073
:106E80002380E700138945006300C7369307000499
:106E90006384F62A232421016FF05FBF930710005B
:106EA00063DE07358327810013877700137787FF19
:106EB000930787002324F100032B47008327070053
:106EC00063560B3E032704001306000493061700C5
:106ED0009795010023AAD56A3387EA009305D0026B
:106EE0002300B700638CC638B307F0403337F00097
:106EF000330B6041938D0700330BEB40930CA000E4
:106F0000130D00006FF09FCB834617001308180085
:106F100013070A006FF0DFC08346170013070A004B
:106F20006FF01FC083270400930600041387170027
:106F300017960100232AE664B387FA00130650026D
:106F40002380C700E314D7B4173703001307878BD8
:106F5000B70610F0130717008347F7FF23A0F6F0DA
:106F6000832704009387F7FF17960100232EF6600E
:106F7000E39207FE6FF09FB1930C0001130D000028
:106F80006FF09FC18327040093060004130A0500D5
:106F900013871700179601002328E65EB387FA00CF
:106FA000130650022380C700E312D7AE1737030041
:106FB00013074785B70610F0130717008347F7FF3D
:106FC00023A0F6F0832704009387F7FF17960100AC
:106FD000232CF65AE39207FE130A05006FF01FAB4D
:106FE0001737030013070782130717008347F7FFBC
:106FF0002320F6F0832704009387F7FF979501007D
:1070000023A4F558E39207FE9386C6FF6FF09FC650
:10701000172703001307077FE39805FC9386C6FF35
:107020006FF05FC5E3FA9DBB930910006FF01FBFBF
:10703000130C000003C70C0093050700E30C07E4E2
:107040009308F0FF1305A00013080004B70610F022
:10705000635E0B0C8327040013861700B387FA00C6
:10706000179301002322C3522380E7006382A508FF
:107070006308060B938C1C0003C70C00130CFCFF69
:1070800093050700E31607FCE35680E1832704001D
:107090009305000213060004B70610F06F00C0004D
:1070A000130CFCFFE3080CDE13871700B387FA000C
:1070B0002380B700179501002328E54C93070700AC
:1070C000E310C7FE172703001307C7731307170042
:1070D0008347F7FF23A0F6F0832704009387F7FF89
:1070E000179501002322F54AE39207FE6FF05FFB3C
:1070F0001727030013070771E30E06F6130717009F
:107100008347F7FF23A0F6F0832704009387F7FF58
:1071100017960100232AF646E39207FE6FF09FF5CB
:10712000172703001307076E6FF05FFD130BFBFFBC
:10713000E3121BF36FF05FF5172703001307876C4B
:10714000B70610F0130717008347F7FF23A0F6F0E8
:10715000832704009387F7FF179601002326F64242
:10716000E39207FE232421016FF05F92979C0100B8
:10717000938C4C2593050B0013850C00EF001050E9
:10718000330CAC40E35880EB832704001306000463
:10719000B70610F06F00C000130CFCFFE30A0CE808
:1071A00013871700B387FA002380770197950100B2
:1071B00023ACE53C93070700E310C7FE1727030045
:1071C00013074764130717008347F7FF23A0F6F060
:1071D000832704009387F7FF9795010023A6F53ACC
:1071E000E39207FE6FF05FFB172703001307876129
:1071F000E39806F4232421016FF05F89832781003F
:107200001387470083A707002324E10013DBF7411E
:107210006FF01FCB172703001307C75EB70610F0E8
:10722000130717008347F7FF23A0F6F08327040016
:107230009387F7FF179601002328F634E39207FEA1
:1072400093071000179701002320F7349307800756
:10725000172703002308F75A6FF09FAF635680018A
:107260009307D002E394FBF0979C0100938C8C155C
:1072700013078002930580026FF09FDC97260300BE
:1072800093864658370610F09386160003C7F6FF1C
:107290002320E6F0032704001307F7FF979501006A
:1072A00023A4E52EE31207FE6FF01FC4938D0700A1
:1072B000930CA000130D00006FF05F90B70710F063
:1072C00023A0A7F26F000000130101FC1303410289
:1072D0002322B10293050300232E11002324C102AF
:1072E0002326D1022328E102232AF102232C0103C1
:1072F000232E110323266100EFF00FF38320C10139
:10730000130500001301010467800000130101FB55
:1073100013038103232481022326A100232CC1020D
:1073200013040500130603001305C10023261102F0
:107330002322F104232ED1022320E104232401057A
:1073400023261105232E6100EFF04F9B8327C100F8
:10735000238007000325C1008320C1023305854037
:10736000032481021301010567800000B70710F0B4
:1073700083A647F403A607F403A747F4E31AD7FE4E
:10738000B7160000938606FAB306D60033B6C600D9
:10739000B305E60023A4D7F423A6B7F46780000062
:1073A000B70710F003A747F403A607F483A647F432
:1073B000E31AD7FEB7160000938606FAB306D60086
:1073C00033B6C60023A4D7F4B305E60023A6B7F46A
:1073D0009307000873A0473067800000130101FF86
:1073E0002324810023261100130440011304F4FF19
:1073F000EF005002E31C04FE8320C100032481003F
:107400001301010167800000130101FF23248100A3
:10741000232611009797010093878717179401007F
:107420001304C41603A70700832704001306F07C87
:1074300093064706938747069795010023AAD5141C
:107440009795010023A4F514634AD6008320C10058
:10745000032481001301010167800000130747899D
:107460009797010023A6E712EF00806C93071000A6
:107470006316F50203270400B71700009387F77619
:1074800013050000E3D4E7FCEFF05FE30324810081
:107490008320C100130101016FB09FB41795010053
:1074A0001305C5F2EFF05FE213052000EFF01FE1D6
:1074B000032481008320C100130101016FB05FB27A
:1074C00017950100130505F26FF01FE017950100F5
:1074D0001305C5F16FF05FDF130101FF2324810065
:1074E0002322910023261100B714000017940100F5
:1074F000130444F093878438130000009387F7FF48
:10750000E39C07FE13050400EFF01FDC6FF09FFE05
:10751000130101FF2326110023248100EF00C0582E
:10752000170700001307C7EB9306000013061000AF
:107530009305200317950100130545ECEFE0CFA953
:1075400013040500EFB05FAC13060500130504003B
:10755000032481008320C10013070000930600006C
:1075600093051000130101016FE00FB9130101FF32
:1075700023261100EF00C05B1307100093070000E3
:10758000631AE5008320C100138507001301010180
:107590006780000017950100130545E3EFF0DFD287
:1075A0008320C10093072000138507001301010108
:1075B00067800000737004306F0000006780000077
:1075C000737004306F000000130101FB232291044B
:1075D00023202105232E3103232C4103B73900003A
:1075E000375AC64137890000B704010023248104BB
:1075F000232A5103232861032326710323248103B3
:107600002320A103232EB101232611042322910359
:10761000232601001305C100179C0100130C4CF92F
:10762000972B0300938B0B22179B0100130BCBF7B7
:10763000179D0100130D0DF7972D0300938D0D2756
:10764000130ADAE6938999031309F9FF130410006A
:107650009384F4FF930A1001930C200093050A0011
:10766000EF105007B307350113D507011797010035
:107670002320F7F49305300033752501EF10D00C6B
:1076800013152500B387AB0003A7C70003A50700A8
:1076900093060000130717001306F0FF9305C100BF
:1076A00023A6E700EF901F916306850097970100DE
:1076B00023A007F28327C1009387170063809706F2
:1076C00003270B002326F1009307170017970100EB
:1076D000232CF7EC63F0FA0683270D0017970100BF
:1076E000232407EC638A8706638A0704639497055B
:1076F000972703009387471B03A5070093051000F6
:10770000EFB04F9F1305800C9797010023AC07E85B
:10771000EFB0DFEC03250C006FF01FF483270B00A4
:10772000232601009387170017970100232EF7E601
:10773000E3E4FAFA03250C006FF05FF203A50D00F5
:1077400093050000EFB00F9B03250C0097970100F5
:1077500023AA87E46FF05FF003A50D0093051000E6
:10776000EFB04F99972703009387071403A50700ED
:1077700093050000EFB00F989307200017970100C2
:107780002322F7E203250C006FF01FED130101FC2B
:1077900013059000232C8102232A91022328210320
:1077A0002326310323244103232E110223225103D4
:1077B00023206103232E7101232C8101232A9101AF
:1077C0002328A10123260100972403009384840722
:1077D000EFA00FEF9797010023A2A7DE1389040003
:1077E000172A0300130ACA0617940100130404DDC4
:1077F00093091000130600009305400013053000A4
:10780000EF900FC22320A900630A052483250400FA
:10781000EFA0CFF7630A35239797010023AA07DA71
:1078200013094900E31849FD03A50400930500006E
:10783000EFA00FFC630605009797010023AA07D865
:107840008325040003A50400EFA08FFA930710001E
:107850006306F5009797010023AC07D603A5040043
:107860009305C1009306000013060000EF908FF40B
:107870008325040003A50400EFA04FF16306050073
:107880009797010023A607D403A5040093060000E0
:10789000130600009305C100EF901FD98325040053
:1078A00003A50400EFA08FEE930710006306F50018
:1078B0009797010023AE07D0032504009305800CA1
:1078C000EFA04FF8630605009797010023A207D0A9
:1078D00097270300938747FD03A50700B70401001E
:1078E0003709FFFFEFB04F9B930710009389E4FF28
:1078F000179C0100130C4CCD179A0100130A4ACDB6
:10790000179701002328F7CA979B0100938B0BCA96
:10791000179D0100130D4DCA130B1000930A500060
:10792000930C6000130919009384F4FF1305000001
:10793000EFA05FEF63080506032504009305F0FF41
:10794000EFA04FF0630A050693060000130600003F
:107950009305C100EF905FCD630665019797010025
:1079600023A807C6EFC05FF48327C10063FCF904B6
:107970003387270163F0EA02130780FF636CF70087
:1079800003270C006374F70EB387E740130730003A
:10799000636AF70C83270A00639807087370043042
:1079A0006F000000032504009305F0FFEFA08FE9AE
:1079B000E31C05F86FF09FF79797010023AA07C013
:1079C0006FF0DFF663F0FA023387F94063FCEC00F6
:1079D00003A70B006376F70AB387E740130730006D
:1079E0006360F70C83270A00639607007370043006
:1079F0006F00000083A70B009387170063FCF90852
:107A00009797010023A407BAEFC05FED83270A0010
:107A1000E39E67F183270D009387170017970100F6
:107A2000232CF7B86FF09FF083270C009387170083
:107A300017970100232AF7B8E39807FC97970100EE
:107A400023A497B86FF05FFC032509008325040089
:107A5000EFA0CFD3E30605DC6FF01FDC73700430BA
:107A60006F000000737004306F000000B307F74030
:107A700013073000E370F7F2737004306F000000FA
:107A8000B307F74013073000E37EF7F47370043058
:107A90006F00000017970100232AF7B06FF0DFF6A0
:107AA000737004306F000000130101FF93080000A1
:107AB0001308000097270300938707DF13071000C0
:107AC00093060000130600409795010093854594A6
:107AD00017050000130585AF23261100232481001C
:107AE000EFA0CFE417240300130404DC8326040072
:107AF000930800001308000097270300938707DB13
:107B00001307100013060040979501009385C59058
:107B1000170500001305C5C7EFA04FE103250400BA
:107B2000032481008320C100130101016FC00FB73E
:107B300097270300938707D1179301001303C3A767
:107B400083A8C70003A6870117970100130747A55D
:107B5000032E03000325070003A8070183A6C7011E
:107B600083A5470103A707023386C8409797010002
:107B7000938707A6832E03003305C54183A707001B
:107B80003336C0003306C040B38606413335A0000B
:107B90003375C500B336D0003307B74017930100E3
:107BA0001303C3A2179601001306469FB306D040E5
:107BB0003337E0009387F7FF032E03000326060008
:107BC0003307E0403375D50093B717003375E500F0
:107BD000B307F040179701002324D79D1727030010
:107BE000232E17C717270300232C07C717270300C7
:107BF000232AB7C63375F500630ACE008327030036
:107C000017970100232CF7986780000013050000E8
:107C100067800000130101FE979701009387879901
:107C2000232E1100232C810003A4070093071000CA
:107C3000630AF4008320C1010324810113010102BE
:107C400067800000979701009387079583A7070037
:107C50001307400693871700636EF7008320C10166
:107C600003248101179701002328F79213010102D1
:107C700067800000979701009387479403A507004A
:107C80009797010023AA0790EFA08FBE630805080D
:107C9000130600009305C100EF905FC163068500E5
:107CA0009797010023A607928327C1003707010099
:107CB0001307E7FF6378F70E3707FFFF1307170077
:107CC0003387E7009306500063F0E616130780FF42
:107CD000979601009386468F636CF71403A70600FE
:107CE0006374F716B387E740130730006372F71425
:107CF000737004306F00000083A70600938717009D
:107D0000179701002322F78C639A0700B707010039
:107D10009387F7FF179701002328F78A179401002C
:107D20001304448783270400930600001306000011
:107D300013972700972703009387C7B0B387E700FF
:107D400003A507009795010093854588EF904FDCC8
:107D500093071000E310F5EE17970100130707874C
:107D600083270700938717009796010023A0F686C4
:107D700083270700639A0700B70701009387F7FF7F
:107D8000179701002324F78483270400130720009A
:107D9000938717006354F7089787010023AC077E89
:107DA0006FF05FE99306500063FAF6023307F7407D
:107DB0009306600063F4E602978601009386067FCF
:107DC00003A70600637CF708B387E740130730007A
:107DD000637AF700737004306F000000978601002B
:107DE0009386C67C978701009387877E83A70700C9
:107DF0006382070283A70600370701001307E7FF26
:107E0000938717006376F7069787010023A0077A08
:107E10006FF0DFF0737004306F000000178701000F
:107E2000232AF7766FF01FE1978601009386C679C3
:107E3000978701009387C77983A70700E39E07EA26
:107E4000737004306F000000B307F7401307300071
:107E5000E370F7FE737004306F000000B307F74063
:107E600013073000E370F7F8737004306F00000000
:107E700017870100232CF7726FF05FEAB305B50096
:107E8000930705006386B70003C707006316070062
:107E90003385A74067800000938717006FF09FFE2F
:107EA000130101FB23229104232C4103232291037C
:107EB000232611042324810423202105232E3103AA
:107EC000232A5103232861032326710323248103DA
:107ED0002320A103232EB101930C0500138A050072
:107EE0009304000063DE05003305A0403337A00093
:107EF000B305B040930C0500338AE5409304F0FFCE
:107F000063DA06003306C040B337C000B306D04082
:107F1000B386F640930A06009389060013840C008A
:107F200013090A0063960628178B0100130B8B3880
:107F30006370CA16B70701006372F6149307F00F57
:107F400063F4C70093098000B3573601330BFB007D
:107F500083470B0013050002B3873701B309F540CF
:107F6000638C0900B3153A01B3D7FC00B31A36018C
:107F700033E9B70033943C0113DB0A0193050B008E
:107F800013050900EF00507C130A050093050B0050
:107F9000939B0A0113050900EF00907693DB0B0118
:107FA0009305050013850B00EF00D072131A0A0128
:107FB00093570401B367FA0063FAA700B387570128
:107FC00063E6570163F4A700B38757013389A740DD
:107FD00093050B0013050900EF001077130A050045
:107FE00093050B0013050900EF00907113140401B1
:107FF00093050500131A0A0113850B00135404019D
:10800000EF00506D33648A00637AA4003304540196
:10801000636654016374A400330454013304A44020
:108020003354340193050000638A04003304804014
:10803000B3378000B305B040B385F54013050400A5
:108040008320C104032481048324410403290104FF
:108050008329C103032A8103832A4103032B0103DC
:10806000832BC102032C8102832C4102032D0102C8
:10807000832DC1011301010567800000B7070001CE
:1080800093090001E362F6EC930980016FF0DFEBE6
:10809000631A06009305000013051000EF005066F8
:1080A000930A0500B707010063FAFA0E9307F00F71
:1080B00063F4570193098000B3D73A01330BFB00F7
:1080C00083470B001305000233095A41B387370178
:1080D000B309F540E38209EAB39A3A01335BFA0047
:1080E000B3153A01B3D7FC0093DB0A0133E9B700BB
:1080F00013050B0093850B00EF001065130A0500B4
:1081000093850B00139C0A0113050B00EF00505FD1
:10811000135C0C019305050013050C00EF00905B48
:10812000131A0A0193570901B367FA0033943C010B
:1081300063FAA700B387570163E6570163F4A7000A
:10814000B3875701338BA74093850B0013050B00B2
:10815000EF00905F130A050093850B0013050B00D9
:10816000EF00105A9305050013050C00EF00905620
:1081700093160901131A0A0193D60601B366DA00B1
:1081800063FAA600B386560163E6560163F4A600BF
:10819000B38656013389A6406FF01FDEB707000192
:1081A00093090001E3EAFAF0930980016FF0DFF030
:1081B0006376DA0093050A006FF01FE7B707010046
:1081C00063FAF604930BF00F33B5DB00131535009B
:1081D00033D7A600978701009387C70DB387E700C1
:1081E00083CB070093050002B38BAB00338B754143
:1081F000631C0B0263E4460163EACC003384CC4089
:10820000B306DA4033B98C0033892641930509005F
:108210006FF09FE1B707000113050001E3EAF6FAEA
:10822000130580016FF0DFFAB3966601335D7601C6
:10823000336DDD00B35D7A01B3156A0133DC7C0177
:1082400013540D01336CBC0013850D00930504001D
:10825000B3196601EF00504F930A0500930504001F
:1082600013850D0033996C01931C0D01EF005049EB
:1082700093DC0C01130A05009305050013850C001F
:10828000EF005045939A0A0113570C0133E7EA00B7
:10829000930D0A00637EA7003307A701930DFAFF31
:1082A0006368A7016376A700930DEAFF3307A70170
:1082B000330AA7409305040013050A00EF00D048D5
:1082C00093050400930A050013050A00EF005043CC
:1082D000930505001304050013850C00EF00903F83
:1082E00093150C01939A0A0193D50501B3E5BA00E1
:1082F0001307040063FEA500B385A5011307F4FF6F
:1083000063E8A50163F6A5001307E4FFB385A501A3
:10831000939D0D01B70C0100B3EDED001384FCFF3C
:10832000B3F78D0033F48900338AA5401385070025
:10833000930504002326F10093DD0D01EF00903931
:1083400093050400930A050013850D00EF00903893
:1083500013DC090193050C002324A10013850D00F3
:10836000EF0050378327C10013040C00930504006D
:10837000130C050013850700EF00D035832681001C
:1083800013D70A013305D5003307A7006374D7005C
:10839000330C9C01B70701009387F7FF9355070142
:1083A0003377F70013170701B3F7FA00B385850198
:1083B000B307F7006366BA00631EBA00637CF90076
:1083C00033863741B3B7C700B385A541B385F540C0
:1083D00093070600B307F9403339F900B305BA40F3
:1083E000B385254133947501B3D767013364F40035
:1083F000B3D565016FF05FC3130101FD2322910224
:10840000232A510123261102232481022320210340
:10841000232E3101232C41012328610123267101E0
:1084200023248101232291012320A101930A050025
:1084300093840500639E0638130406009309050023
:1084400017890100130909E763F8C512B70701008E
:10845000138B05006378F6101307F00F3337C7004E
:1084600013173700B357E6003309F90083460900B4
:108470003387E60093060002B386E640638C06006D
:10848000B394D40033D7EA003314D600336B97008B
:10849000B399DA00935A040193850A0013050B007F
:1084A000EF00902A1309050093850A00931B04012D
:1084B00013050B00EF00D02493DB0B0193040500A0
:1084C0009305050013850B00EF00D0201319090157
:1084D00093D70901B367F900138A040063FEA7006C
:1084E000B3878700138AF4FF63E8870063F6A70069
:1084F000138AE4FFB3878700B384A74093850A00FB
:1085000013850400EF0050241309050093850A0029
:1085100013850400EF00D01E939909019304050010
:10852000930505001319090113850B0093D909015F
:10853000EF00501AB36939011386040063FCA900E7
:10854000B30934011386F4FF63E6890063F4A900DC
:108550001386E4FF13140A013364C400130A0000F5
:108560006F000013B707000113070001E36CF6EE7C
:10857000130780016FF01FEF138A0600631A0600CD
:108580009305000013051000EF0090171304050079
:10859000B7070100637EF4129307F00F63F48700BE
:1085A000130A8000B35744013309F9000347090057
:1085B0009306000233074701B386E6406394061230
:1085C000B3848440130A1000135B040193050B006D
:1085D00013850400EF0050171309050093050B00E5
:1085E00013850400931B0401EF00901193DB0B0132
:1085F000930405009305050013850B00EF00900D13
:108600001319090193D70901B367F900938A04008C
:1086100063FEA700B3878700938AF4FF63E88700AF
:1086200063F6A700938AE4FFB3878700B384A7406B
:1086300093050B0013850400EF00101113090500CA
:1086400093050B0013850400EF00900B939909012B
:1086500093040500930505001319090113850B0008
:1086600093D90901EF001007B3693901138604009B
:1086700063FCA900B30934011386F4FF63E68900A3
:1086800063F4A9001386E4FF13940A013364C40061
:108690001305040093050A008320C102032481020C
:1086A00083244102032901028329C101032A810194
:1086B000832A4101032B0101832BC100032C81007C
:1086C000832C4100032D010013010103678000008A
:1086D000B7070001130A0001E366F4EC130A8001F6
:1086E0006FF05FEC3314D40033DAE400B399DA00AE
:1086F00033D7EA00935A0401B394D40093850A0057
:1087000013050A00336B9700EF00100413090500EE
:1087100093850A0013050A00931B0401EF00407EB5
:1087200093DB0B01930405009305050013850B00F3
:10873000EF00407A1319090113570B013367E90061
:10874000138A0400637EA70033078700138AF4FFAF
:10875000636887006376A700138AE4FF3307870006
:10876000B304A74093850A0013850400EF00C07D81
:108770001309050093850A0013850400EF00407873
:10878000930405009305050013850B00EF0080742A
:1087900013170B011357070113190901B367E900F8
:1087A0001387040063FEA700B38787001387F4FFD5
:1087B00063E8870063F6A7001387E4FFB3878700A9
:1087C000131A0A01B384A740336AEA006FF0DFDFAF
:1087D00063ECD51EB707010063F4F6041307F00F2E
:1087E000B335D7009395350033D7B600978701008E
:1087F000938747ACB387E70003C70700130A00025B
:108800003307B700330AEA4063160A021304100064
:10881000E3E096E833B6CA00134416006FF05FE752
:10882000B707000193050001E3E0F6FC9305800122
:108830006FF09FFBB35CE600B3964601B3ECDC003F
:1088400033D4E40093DB0C01B397440133D7EA003F
:1088500093850B0013050400336BF700B319460131
:10886000EF00806E1309050093850B0013050400CB
:10887000139C0C01EF00C068135C0C01930405000D
:108880009305050013050C00EF00C06413190901DE
:1088900013570B013367E90013840400637EA700BC
:1088A000330797011384F4FF636897016376A70089
:1088B0001384E4FF33079701B304A74093850B00AB
:1088C00013850400EF0040681309050093850B0031
:1088D00013850400EF00C0629304050093050500B2
:1088E00013050C00EF00005F93170B01131909012A
:1088F00093D70701B367F9001386040063FEA7004E
:10890000B38797011386F4FF63E8970163F6A70026
:108910001386E4FFB387970113140401B70B01001A
:108920003364C4001389FBFF337D240133F929012B
:10893000B384A7409305090013050D00EF0080598B
:10894000935C040193050900130B050013850C00CB
:10895000EF00405893D90901130C050093850900D5
:1089600013850C00EF0000571309050093850900DB
:1089700013050D00EF0000563305850193570B01D9
:108980003385A70063748501330979019357050185
:10899000B387270163E6F402E392F4BCB707010052
:1089A0009387F7FF3375F50013150501337BFB0043
:1089B00033964A0133056501130A0000E37AA6CC19
:1089C0001304F4FF6FF09FB9130A000013040000B2
:1089D0006FF01FCC130101FB232481042322910497
:1089E000232E310323229103232611042320210562
:1089F000232C4103232A51032328610323267103D7
:108A0000232481032320A103232EB101930C05000D
:108A1000938905001304050093840500639E0626D0
:108A200013090600138A0600978A0100938A8A8830
:108A300063F4C514B70701006376F6129307F00FCD
:108A400063F4C700130A8000B3574601B38AFA00E3
:108A500003C70A001305000233074701330AE54044
:108A6000630C0A00B395490133D7EC003319460172
:108A7000B364B70033944C01935A090193850A00FB
:108A800013850400EF00404C9309050093850A000C
:108A9000131B090113850400EF008046135B0B01D3
:108AA0009305050013050B00EF00C04293990901DF
:108AB00093570401B3E7F90063FAA700B3872701CE
:108AC00063E6270163F4A700B3872701B384A740B7
:108AD00093850A0013850400EF0000479309050001
:108AE00093850A0013850400EF00804113140401EC
:108AF000930505009399090113050B001354040114
:108B0000EF00403D33E48900637AA400330424017C
:108B1000636624016374A400330424013304A44075
:108B200033554401930500008320C10403248104CC
:108B300083244104032901048329C103032A8103F7
:108B4000832A4103032B0103832BC102032C8102DF
:108B5000832C4102032D0102832DC1011301010564
:108B600067800000B7070001130A0001E36EF6EC0E
:108B7000130A80016FF05FED631A06009305000091
:108B800013051000EF00C03713090500B7070100F7
:108B9000637AF90E9307F00F63F42701130A80003C
:108BA000B3574901B38AFA0003C70A00130500024C
:108BB000B384294133074701330AE540E30E0AEA4B
:108BC00033194901B3DAE900B395490133D7EC0011
:108BD00093540901336BB70013850A009385040091
:108BE000EF0080369309050093850400931B09016B
:108BF00013850A00EF00C03093DB0B0193050500DD
:108C000013850B00EF00002D9399090193570B0179
:108C1000B3E7F90033944C0163FAA700B387270147
:108C200063E6270163F4A700B3872701B38AA7404F
:108C30009385040013850A00EF00003193090500B5
:108C40009385040013850A00EF00802B930505002F
:108C500013850B00EF00002893150B019399090170
:108C600093D50501B3E5B90063FAA500B3852501E5
:108C700063E6250163F4A500B3852501B384A5400F
:108C80006FF09FDFB7070001130A0001E36AF9F0F4
:108C9000130A80016FF0DFF0E3E8D5E8B7070100C1
:108CA00063FCF604930BF00F33B5DB0013153500AE
:108CB00033D7A600977701009387C75FB387E70094
:108CC00083CB070093050002B38BAB00338B754158
:108CD000631E0B0263E4360163EACC003384CC40AC
:108CE000B386D94033B58C00B384A6401305040085
:108CF000938504006FF05FE3B707000113050001DF
:108D0000E3E8F6FA130580016FF09FFAB396660167
:108D1000335D7601336DDD0033D47901B39569019C
:108D200033DC7C0193540D01336CBC00130504004B
:108D300093850400B31A6601EF000021130A0500B1
:108D4000938504001305040033996C01931C0D01F5
:108D5000EF00001B93DC0C011304050093050500D4
:108D600013850C00EF000017131A0A0113570C01AA
:108D70003367EA00130A0400637EA7003307A701E4
:108D8000130AF4FF6368A7016376A700130AE4FFE0
:108D90003307A701B309A740938504001385090091
:108DA000EF00801A93850400130405001385090061
:108DB000EF000015930505009304050013850C00D2
:108DC000EF00401193150C011314040193D5050114
:108DD000B365B4001387040063FEA500B385A50145
:108DE0001387F4FF63E8A50163F6A5001387E4FF8A
:108DF000B385A501131A0A01B70C0100336AEA0012
:108E00001384FCFFB3778A0033F48A00B384A5404F
:108E100013850700930504002326F100135A0A0165
:108E2000EF00400B930905009305040013050A00A9
:108E3000EF00400A13DC0A01930D050093050C00B6
:108E400013050A00EF0000098327C100130A05007B
:108E500093050C0013850700EF00C0073305B5012B
:108E600013D709013307A7006374B701330A9A01C6
:108E7000B70701009387F7FF935507013377F70092
:108E800013170701B3F7F900B3854501B307F700DE
:108E900063E6B400639EB400637CF90033865741F7
:108EA000B3B7C700B385A541B385F5409307060066
:108EB000B307F9403339F900B385B440B385254190
:108EC00033947501B3D767013365F400B3D56501F9
:108ED0006FF09FC5130605001305000093F61500FB
:108EE000638406003305C50093D5150013161600DC
:108EF000E39605FE678000006340050663C605062D
:108F000013860500930505001305F0FF630C0602A8
:108F100093061000637AB6006358C000131616005B
:108F200093961600E36AB6FE1305000063E6C500DB
:108F3000B385C5403365D50093D616001356160089
:108F4000E39606FE6780000093820000EFF05FFB6F
:108F500013850500678002003305A04063D8050033
:108F6000B305B0406FF0DFF9B305B0409382000065
:108F7000EFF01FF93305A0406780020093820000E4
:108F800063CA0500634C0500EFF09FF713850500E9
:108F900067800200B305B040E35805FE3305A040EA
:108FA000EFF01FF63305B0406780020097770100AD
:108FB0009387075B83A607001777010013070759FC
:108FC0000327070023A2A600637EE50017770100B0
:108FD000130787580325070083A5070093854500DD
:108FE0006F704FFA130101FF232481002326110023
:108FF00017770100130787561304050003250700A0
:1090000083A5070093854500EF70CFF797770100A0
:109010009387075283A707006376F40097770100D0
:1090200023A887508320C10003248100130101017C
:1090300067800000977701009387875203A7070096
:1090400083A60700832747049387F7FF2322F704AB
:1090500083A74604639407007360043067800000B0
:10906000130101FE232C8100232A91001304050023
:109070009384050023282101232631012324410163
:1090800023225101232E1100EF909FF68327040025
:1090900003290401B7090001B3E59700930AC4004E
:1090A0002320B400930400009389F9FF370A0002DB
:1090B0000327040063822A0503260900130509001B
:1090C000B3654701B37636019317560033F7E600D0
:1090D0000329490063C60700631607006FF05FFDB0
:1090E000E398E6FC9317760063D40700B3E4D4005A
:1090F000EFB04FB86FF0DFFB93C4F4FFB3F4E400BC
:1091000023209400EFA04FA2032504008320C10177
:109110000324810183244101032901018329C10022
:10912000032A8100832A41001301010267800000A5
:10913000130101FF2326110023248100EFE04FBD1E
:1091400017E7FFFF1307872C930600001306100094
:1091500093054006177501001305C52AEFC0CFE738
:109160006302050213040500EF901FEA13060500D1
:109170001307000093060000930510001305040078
:10918000EFC08FF7EF901FB48320C100032481004C
:0C919000130500001301010167800000BE
:02000004800278
:10000000F467FEFF6469FEFF0068FEFF6469FEFF9F
:100010006469FEFF6469FEFF6469FEFF2868FEFFF5
:100020006469FEFF6469FEFF5068FEFF6068FEFFC2
:100030006469FEFF7868FEFF8868FEFF8868FEFF3F
:100040008868FEFF8868FEFF8868FEFF8868FEFFFC
:100050008868FEFF8868FEFF8868FEFF6469FEFF0F
:100060006469FEFF6469FEFF6469FEFF6469FEFF68
:100070006469FEFF6469FEFF6469FEFF6469FEFF58
:100080006469FEFF6469FEFF6469FEFF6469FEFF48
:100090006469FEFF6469FEFF6469FEFF6469FEFF38
:1000A0006469FEFF6469FEFF6469FEFF6469FEFF28
:1000B0006469FEFF6469FEFF6469FEFF6469FEFF18
:1000C0006469FEFF6469FEFF6469FEFF6469FEFF08
:1000D0006469FEFF6469FEFF6469FEFF6469FEFFF8
:1000E0006469FEFF6469FEFF6469FEFF6469FEFFE8
:1000F0006469FEFF6469FEFF6469FEFF6469FEFFD8
:10010000CC68FEFFF468FEFF6469FEFF6469FEFFD1
:100110006469FEFF6469FEFF6469FEFF6469FEFFB7
:100120006469FEFF5469FEFF6469FEFF6469FEFFB7
:100130000466FEFF0C67FEFF6469FEFF6469FEFF54
:100140005C67FEFF6469FEFFD467FEFF6469FEFF23
:100150006469FEFF1C68FEFFC06DFEFF2C6EFEFF93
:10016000CC6DFEFF2C6EFEFF2C6EFEFF2C6EFEFF94
:100170002C6EFEFF646CFEFF2C6EFEFF2C6EFEFFED
:100180008C6CFEFF9C6CFEFF2C6EFEFFB46CFEFFC1
:10019000C46CFEFFC46CFEFFC46CFEFFC46CFEFFAB
:1001A000C46CFEFFC46CFEFFC46CFEFFC46CFEFF9B
:1001B000C46CFEFF2C6EFEFF2C6EFEFF2C6EFEFF4D
:1001C0002C6EFEFF2C6EFEFF2C6EFEFF2C6EFEFFD3
:1001D0002C6EFEFF2C6EFEFF2C6EFEFF2C6EFEFFC3
:1001E0002C6EFEFF2C6EFEFF2C6EFEFF2C6EFEFFB3
:1001F0002C6EFEFF2C6EFEFF2C6EFEFF2C6EFEFFA3
:100200002C6EFEFF2C6EFEFF2C6EFEFF2C6EFEFF92
:100210002C6EFEFF2C6EFEFF2C6EFEFF2C6EFEFF82
:100220002C6EFEFF2C6EFEFF2C6EFEFF2C6EFEFF72
:100230002C6EFEFF2C6EFEFF2C6EFEFF2C6EFEFF62
:100240002C6EFEFF2C6EFEFF2C6EFEFF2C6EFEFF52
:100250002C6EFEFF2C6EFEFF086DFEFF446DFEFF50
:100260002C6EFEFF2C6EFEFF2C6EFEFF2C6EFEFF32
:100270002C6EFEFF2C6EFEFF2C6EFEFFB06DFEFF9F
:100280002C6EFEFF2C6EFEFF386AFEFF8C6BFEFFAD
:100290002C6EFEFF2C6EFEFF1C6CFEFF2C6EFEFF14
:1002A000486CFEFF2C6EFEFF2C6EFEFF206EFEFFE4
:1002B000000102020303030304040404040404040D
:1002C00005050505050505050505050505050505DE
:1002D00006060606060606060606060606060606BE
:1002E00006060606060606060606060606060606AE
:1002F000070707070707070707070707070707078E
:10030000070707070707070707070707070707077D
:10031000070707070707070707070707070707076D
:10032000070707070707070707070707070707075D
:10033000080808080808080808080808080808083D
:10034000080808080808080808080808080808082D
:10035000080808080808080808080808080808081D
:10036000080808080808080808080808080808080D
:1003700008080808080808080808080808080808FD
:1003800008080808080808080808080808080808ED
:1003900008080808080808080808080808080808DD
:1003A00008080808080808080808080808080808CD
:1003B000546D725100000000546D7220537663003A
:1003C000286E756C6C2900004572726F7220696E20
:1003D00020787878207461736B73200D0A00000018
:1003E0006D69616F750A00006D69616F75320A0091
:1003F00068756E6772790A0054696D657232000023
:10040000436865636B54696D65720000536574548D
:0C04100078000000536574527800000072
:10041C001000000000000000017A5200017C010174
:10042C001B0D02005000000018000000687AFEFF4F
:10043C005805000000440E507489039406990B81F2
:10044C0001880292049305950796089709980A9AD1
:10045C000C9B0D036C010AC144C844C944D244D35B
:10046C0044D444D544D644D744D844D944DA44DBA4
:10047C00440E00440B0000004C0000006C00000017
:10048C006C7FFEFFDC05000000440E307089039584
:10049C00078101880292049305940696089709989F
:1004AC000A990B9A0C0370020AC144C844C944D27D
:1004BC0044D344D444D544D644D744D844D944DA5C
:1004CC00440E00440B00000050000000BC00000073
:1004DC00F884FEFF0005000000440E507488028969
:1004EC00039305990B81019204940695079608973E
:1004FC0009980A9A0C9B0D0320010AC144C844C9EF
:10050C0044D244D344D444D544D644D744D844D913
:0C051C0044DA44DB440E00440B000000F5
:1005BC00FC8F010009000000FFFF0000FFFF00009E
:0405CC00010000002A
:040000058000004037
:00000001FF
